:020000040800F2
:1000000000090020D5040008C12800084128000884
:1000100099280008412800086D280008D704000826
:10002000D7040008D7040008D7040008613A000884
:10003000D7040008D7040008D7040008D704000834
:10004000D7040008D7040008D7040008D704000824
:10005000D7040008D704000885640008AD640008D0
:10006000D5640008FD64000825650008D704000871
:10007000D7040008D7040008D7040008D7040008F4
:10008000D7040008D7040008D70400088524000816
:10009000B1240008C1240008D70400084D650008F9
:1000A000D7040008D7040008D7040008D7040008C4
:1000B00035660008D7040008D7040008D7040008F4
:1000C000D7040008D7040008D7040008D7040008A4
:1000D000D704000821660008D7040008D7040008E8
:1000E000B1650008D7040008D7040008D704000849
:1000F000D7040008D7040008D7040008D704000874
:10010000D7040008D7040008D7040008D704000863
:10011000D7040008D7040008D7040008D704000853
:10012000D7040008D7040008D7040008D704000843
:10013000D7040008D7040008D7040008D704000833
:10014000D7040008D7040008D7040008E55A0008BF
:10015000D7040008D7040008D7040008D704000813
:10016000D7040008D7040008D7040008D704000803
:10017000D7040008D7040008D7040008D7040008F3
:10018000D7040008D7040008D7040008D7040008E3
:10019000D7040008D7040008D7040008D7040008D3
:1001A000D7040008D7040008D7040008D7040008C3
:1001B000D7040008D7040008D7040008D7040008B3
:1001C0005D160008000000000000000000000000B4
:1001D00053B94AB9002908BF00281CBF4FF0FF31AE
:1001E0004FF0FF3000F074B9ADF1080C6DE904CEAA
:1001F00000F006F8DDF804E0DDE9022304B0704702
:100200002DE9F047089D04468E46002B4DD18A42C9
:10021000944669D9B2FA82F252B101FA02F3C2F1FC
:10022000200120FA01F10CFA02FC41EA030E94408D
:100230004FEA1C48210CBEFBF8F61FFA8CF708FBAE
:1002400016E341EA034306FB07F199420AD91CEB86
:10025000030306F1FF3080F01F81994240F21C81B8
:10026000023E63445B1AA4B2B3FBF8F008FB103300
:1002700044EA034400FB07F7A7420AD91CEB040435
:1002800000F1FF3380F00A81A74240F20781644405
:10029000023840EA0640E41B00261DB1D44000238A
:1002A000C5E900433146BDE8F0878B4209D9002DEE
:1002B00000F0EF800026C5E9000130463146BDE878
:1002C000F087B3FA83F6002E4AD18B4202D38242E2
:1002D00000F2F980841A61EB030301209E46002D91
:1002E000E0D0C5E9004EDDE702B9FFDEB2FA82F2E6
:1002F000002A40F09280A1EB0C014FEA1C471FFA44
:100300008CFE0126200CB1FBF7F307FB131140EA2A
:1003100001410EFB03F0884208D91CEB010103F1F7
:10032000FF3802D2884200F2CB804346091AA4B2B9
:10033000B1FBF7F007FB101144EA01440EFB00FE8D
:10034000A64508D91CEB040400F1FF3102D2A645F2
:1003500000F2BB800846A4EB0E0440EA03409CE791
:10036000C6F12007B34022FA07FC4CEA030C20FA3E
:1003700007F401FA06F31C43F9404FEA1C4900FA5E
:1003800006F3B1FBF9F8200C1FFA8CFE09FB1811DB
:1003900040EA014108FB0EF0884202FA06F20BD94E
:1003A0001CEB010108F1FF3A80F08880884240F29E
:1003B0008580A8F102086144091AA4B2B1FBF9F0E2
:1003C00009FB101144EA014100FB0EFE8E4508D9DD
:1003D0001CEB010100F1FF346CD28E456AD9023862
:1003E000614440EA0840A0FB0294A1EB0E01A14247
:1003F000C846A64656D353D05DB1B3EB080261EBB5
:100400000E0101FA07F722FA06F3F1401F43C5E98E
:10041000007100263146BDE8F087C2F12003D840C4
:100420000CFA02FC21FA03F3914001434FEA1C4706
:100430001FFA8CFEB3FBF7F007FB10360B0C43EAF8
:10044000064300FB0EF69E4204FA02F408D91CEBA8
:10045000030300F1FF382FD29E422DD902386344A6
:100460009B1B89B2B3FBF7F607FB163341EA034146
:1004700006FB0EF38B4208D91CEB010106F1FF3895
:1004800016D28B4214D9023E6144C91A46EA00468C
:1004900038E72E46284605E70646E3E61846F8E61E
:1004A0004B45A9D2B9EB020864EB0C0E0138A3E767
:1004B0004646EAE7204694E74046D1E7D0467BE748
:1004C000023B614432E7304609E76444023842E7C0
:1004D000704700BF02E000F000F8FEE772B63A484D
:1004E00080F30888394880F3098839484EF6085166
:1004F000CEF20001086040F20000CCF200004EF69F
:100500003471CEF200010860BFF34F8FBFF36F8FDD
:1005100040F20000C0F2F0004EF68851CEF2000129
:100520000860BFF34F8FBFF36F8F4FF00000E1EE15
:10053000100A4EF63C71CEF200010860062080F3EE
:100540001488BFF36F8F04F0B1FF04F08DFF05F046
:100550002FFE4FF055301F491B4A91423CBF41F8D6
:10056000040BFAE71C49194A91423CBF41F8040BBD
:10057000FAE71A491A4A1B4B9A423EBF51F8040B3C
:1005800042F8040BF8E700201749184A91423CBF93
:1005900041F8040BFAE704F06BFF05F055FE144C2C
:1005A000144DAC4203DA54F8041B8847F9E700F015
:1005B00041F8114C114DAC4203DA54F8041B884742
:1005C000F9E704F053BF00000009002000110020EB
:1005D000000000080001002000090020506D000804
:1005E00000110020C4110020C8110020D43F0020B9
:1005F000C0010008C4010008C4010008C4010008CB
:100600002DE9F04F2DED108AC1F80CD0C3689D463E
:10061000BDEC108ABDE8F08F002383F311882846D3
:10062000A047002004F0D0FAFEE704F03FFA00DF14
:10063000FEE70000F8B504F0CDFE074604F00AFF1F
:100640000546B8BB204B9F4234D001339F4234D083
:100650001E4B27F0FF029A4232D1F8B200F050FE52
:100660002E4642F2107400F051FE08B100242646D6
:1006700002F044FA20B1032000F07CF80024264662
:1006800035B1134B9F4203D004F0DCFE0024264614
:10069000002004F0A9FE0EB100F082F801F080F90C
:1006A00000F058FE01F056F8204600F0D9F800F0AE
:1006B00077F8F9E72E460024D5E704460126D2E76D
:1006C00006464FF47A74CEE7010007B0000008B088
:1006D000263A09B008B501F009F8A0F12003584204
:1006E000584108BD07B541F21203022101A8ADF837
:1006F000043001F019F803B05DF804FB38B520238D
:1007000083F311881748C3680BB104F0E3FA164A63
:10071000144800234FF47A7104F0A0FA002383F305
:100720001188124C236813B12368013B236063686E
:1007300013B16368013B63600D4D2B7833B9636877
:100740007BB9022001F0A6F8322363602B78032BDB
:1007500007D163682BB9022001F09CF84FF47A733B
:10076000636038BDC8110020FD060008E4120020B7
:10077000DC110020084B187003280CD8DFE800F0CB
:1007800008050208022001F07BB8022001F070B8D1
:10079000024B00225A607047DC110020E412002056
:1007A00010B502F0ABF930B1274B03221A70274B7A
:1007B00000225A6010BD264B264A1C46196801319A
:1007C000F8D004339342F9D16268A242F2D3224BAB
:1007D0009B6803F1006303F520439A42EAD204F0D8
:1007E00017FE002000F0D0FF0220FFF7C3FF1B4BD5
:1007F0009A6D00229A65996F9A67996FD96DDA653B
:10080000D96FDA67D96F196E1A66D3F88010C3F8FA
:100810008020D3F88020DA6A42F48052DA62DA6A01
:1008200022F48052DA62DB6A72B64FF0E0232021B4
:10083000C3F8084DD4E9003281F311889D4683F353
:1008400008881047B6E700BFDC110020E412002042
:1008500000A0000820A000080011002000100240A5
:100860002DE9F04F93B0AC4B00902022FF210AA855
:100870009D6801F03FF8A94A1378A3B9A84801215F
:10088000C3601170202383F31188C3680BB104F097
:1008900021FAA44AA24800234FF47A7104F0DEF949
:1008A000002383F31188009B13B19F4B009A1A60B9
:1008B0009E4A009C1378032B1EBF002313709A4A94
:1008C0004FF0000A18BF5360D3465646D146012068
:1008D00000F0D6FF24B1944B1B68002B00F015826A
:1008E000002000F003FF0390039B002B01DA00F0CF
:1008F00079FD039B002BEDDB012000F0B9FF039B8A
:10090000213B162BE3D801A252F823F06909000815
:1009100091090008250A0008CF080008CF08000840
:10092000CF080008AF0A00087F0C0008990B0008E8
:10093000FB0B0008230C0008490C0008CF08000836
:100940005B0C0008CF080008CD0C0008090A00085D
:10095000CF080008110D000875090008090A0008F1
:10096000CF080008FB0B00080220FFF7B3FE0028A9
:1009700040F0F581009B0221BAF1000F08BF1C4630
:1009800005A841F21233ADF8143000F0CDFE9EE719
:100990004FF47A7000F0AAFE071EEBDB0220FFF78F
:1009A00099FE0028E6D0013F052F00F2DA81DFE84A
:1009B00007F0030A0D10133605230593042105A83B
:1009C00000F0B2FE17E054480421F9E7584804212A
:1009D000F6E758480421F3E74FF01C08404600F0C2
:1009E000D5FE08F104080590042105A800F09CFE3E
:1009F000B8F12C0FF2D1012000FA07F747EA0B0BF0
:100A00005FFA8BFB4FF0000900F0C0FF26B10BF03E
:100A10000B030B2B08BF0024FFF764FE57E7464883
:100A20000421CDE7002EA5D00BF00B030B2BA1D199
:100A30000220FFF74FFE074600289BD0012000F060
:100A4000A3FE0220FFF796FE00265FFA86F84046D6
:100A500000F0AAFE044690B10021404600F0B4FE2A
:100A600001360028F1D1BA46044641F212130221A0
:100A700005A8ADF814303E4600F056FE27E70120E9
:100A8000FFF778FE2546244B9B68AB4207D92846E2
:100A900000F07CFE013040F067810435F3E7234B22
:100AA00000251D70204BBA465D603E46ACE7002E27
:100AB0003FF460AF0BF00B030B2B7FF45BAF022016
:100AC000FFF758FE322000F011FEB0F10008FFF6EB
:100AD00051AF18F003077FF44DAF0F4A926808EB4F
:100AE000050393423FF646AFB8F5807F3FF742AF2C
:100AF000124B0193B84523DD4FF47A7000F0F6FDF8
:100B00000390039A002AFFF635AF019B039A03F87E
:100B1000012B0137EDE700BF00110020E01200209B
:100B2000C8110020FD060008E4120020DC1100209E
:100B300004110020081100200C110020E0110020F9
:100B4000C820FFF7C7FD074600283FF413AF1F2D4D
:100B500011D8C5F1200242450AAB25F0030028BF99
:100B6000424683490192184400F09EFE019A804853
:100B7000FF2100F0BFFE4FEAA8037D490193C8F3AF
:100B80008702284600F0BEFE064600283FF46DAFFF
:100B9000019B05EB830537E70220FFF79BFD00284B
:100BA0003FF4E8AE00F02EFE00283FF4E3AE00274D
:100BB000B846704B9B68BB4218D91F2F11D80A9BAF
:100BC00001330ED027F0030312AA134453F8203C3C
:100BD00005934046042205A901F07AFF04378046B8
:100BE000E7E7384600F0D2FD0590F2E7CDF8148033
:100BF000042105A800F098FD06E70023642104A85D
:100C0000049300F087FD00287FF4B4AE0220FFF7C4
:100C100061FD00283FF4AEAE049800F0E9FD0590B8
:100C2000E6E70023642104A8049300F073FD002884
:100C30007FF4A0AE0220FFF74DFD00283FF49AAEEE
:100C4000049800F0D7FDEAE70220FFF743FD0028F3
:100C50003FF490AE00F0E6FDE1E70220FFF73AFD39
:100C600000283FF487AE05A9142000F0E1FD04211F
:100C70000746049004A800F057FD3946B9E7322032
:100C800000F034FD071EFFF675AEBB077FF472AEB1
:100C9000384A926807EB090393423FF66BAE022095
:100CA000FFF718FD00283FF465AE27F003074F4417
:100CB000B9453FF4A9AE484600F068FD042105900F
:100CC00005A800F031FD09F10409F1E74FF47A704D
:100CD000FFF700FD00283FF44DAE00F093FD002823
:100CE00044D00A9B01330BD008220AA9002000F04F
:100CF00009FE00283AD02022FF210AA800F0FAFDC0
:100D0000FFF7F0FC1C4803F065FF13B0BDE8F08F5F
:100D1000002E3FF42FAE0BF00B030B2B7FF42AAE0B
:100D20000023642105A8059300F0F4FC0746002881
:100D30007FF420AE0220FFF7CDFC804600283FF470
:100D400019AEFFF7CFFC41F2883003F043FF05985E
:100D500000F066FE464600F019FE3C46B7E5064642
:100D600052E64FF0000905E6BA467EE637467CE6D5
:100D7000E011002000110020A0860100094A13683C
:100D800049F2690099B21B0C00FB01331360064B5A
:100D9000186844F2506182B2000C01FB0200186036
:100DA00080B27047141100201011002010B50021EE
:100DB0001022044600F09EFD034B03CB20606160CF
:100DC0001868A06010BD00BF9075FF1F2DE9F041AD
:100DD000ADF54E7D0DF134086CAC40F2751207464E
:100DE0000D460EA80021C8F8001000F083FD4FF456
:100DF000C4720021204600F07DFD01F069FD254B05
:100E00004FF47A72B0FBF2F0186093E80700012308
:100E100084E807000DF5E9702382FFF7C7FF41F270
:100E200004731D49238406A805F0C8FD192384F81E
:100E300032310DF2E32206AB0DF1300C1E4603CE2B
:100E4000664510605160334602F10802F6D13378EE
:100E5000137041460122204601F040FD0023039318
:100E6000AB7E029305F11903019380B20123CDE912
:100E700004800093E97E05A3D3E90023384602F0FD
:100E800095F90DF54E7DBDE8F08100BF9E6AC42145
:100E9000818A46EEEC120020EC6900082DE9F0434F
:100EA000224DBBB001F014FDAB6840F2ED22C31A35
:100EB000934232D906AFA8602B462822002138463B
:100EC00002F05CFB05F10E0000F00CFD002604466C
:100ED0005FFA80F905F10E08F3B2F100994501F1CE
:100EE000280107D908EB06030822384602F046FB22
:100EF0000136F1E708230122CDE9023205340C4B1B
:100F00000193A4B230230093CDE9047405A3D3E97F
:100F10000023297B074802F049F93BB0BDE8F08384
:100F2000AFF3008078F6339F93CACD8D0034002054
:100F30000D34002004230020F0B58B8A013B9BB2C6
:100F4000C92BC9B006460C4647D8274D2F7B27BB77
:100F500005F10C03009308223B463946204602F077
:100F6000D1F97B1CFAB2D9001F46A38A013B9A42F1
:100F700005DA0E322A44009200230822EEE700230D
:100F80000022C5E900230023AB6085F8D730C5F8FF
:100F9000D8302B7B0BB9E37E2B738122002106AD69
:100FA00027A800F0A7FC0122294627A801F064FD2C
:100FB00000230393A37E029304F1190380B20193EB
:100FC0002823CDE90450E17E0093304604A3D3E901
:100FD000002302F0EBF8FFF761FF49B0F0BD00BF5E
:100FE00026417272DF25D7B70034002070B50D4658
:100FF00014461E4602F070F850B9022E10D1012C92
:101000000ED112A3D3E90023C5E90023012007E094
:10101000282C10D005D8012C09D0052C0FD0002089
:1010200070BD302CFBD10BA3D3E90023ECE70BA35D
:10103000D3E90023E8E70BA3D3E90023E4E70BA3FC
:10104000D3E90023E0E700BFAFF30080401DA120FB
:1010500026812A0B78F6339F93CACD8D9E6AC421D0
:10106000818A46EE26417272DF25D7B7F017304AE3
:1010700039059E562DE9F04F8DB002AF80460D46E2
:1010800002F02AF8044600285CD12B7E022B1BD1EB
:10109000EB8A012B18D101F01BFC0646FFF76EFE10
:1010A00003464FF4C870DFF81C92B3FBF0F206F56C
:1010B000167602FB103316FA83F3C9F80030EB7E84
:1010C00033B97B4B00221A702C37BD46BDE8F08F38
:1010D000AB8AE6B2013BB34204F101040CD907F13B
:1010E00008031E44E10000960023082201F0F801E5
:1010F000284602F007F9EBE707F11800FFF756FE64
:10110000324607F1180107F1080005F02BFB002813
:10111000D7D10F2E08D8664B1E70D9F80030A3F532
:101120001673C9F80030CFE7FB1DF8710146009334
:1011300007220346284602F0E5F8F979404601F017
:10114000C3FFC1E7EB8A282B26D010D8012B1ED075
:10115000052BB9D1BFF34F8F5649574BCA6802F4DC
:10116000E0621343CB60BFF34F8F00BFFDE7302B2E
:10117000AAD16B7E514C0133627BDBB29342E946CC
:1011800003D1EA7E237B9A420BD0CD469CE72946C9
:101190004046FFF71BFE97E729464046FFF7CCFE87
:1011A00092E74FF0000807F11803A7F81880102203
:1011B000009341460123284602F0A4F8AE8A023E7D
:1011C000B6B2F31C9B109B000733DB08A9EBC303EB
:1011D0009D460DF1080A1FFA88F34FEAC8019E42A6
:1011E00001F110010AD90AEB080300930822002339
:1011F000284602F087F808F10108ECE794F8D700D8
:1012000000F0D2FAD4F8D810054619B994F8D700EE
:1012100000F0DAFAD4F8D83033449D4205D294F87D
:10122000D7000021013000F0CFFA4FEA960B4FF0C3
:1012300000081FFA88F18B45D4E9003209D90AEB7E
:10124000880103EB8800012200F05CFB08F1010833
:10125000EFE7F31842F10002C4E90032D4F8D830C5
:1012600094F8D70006EB0308C4F8D88000F09CFA85
:10127000804509D394F8D730D4F8D8000133401B07
:1012800084F8D730C4F8D800FF2E0D4D09D80023BC
:10129000237300F0B7FA01F031FC288108B9FFF799
:1012A0007FFA23689B0A01332B810023A3606CE73C
:1012B000FD22002000ED00E00400FA0500340020CB
:1012C000EC1200200023002010B50A4B0A4A1A60D5
:1012D00003F5805393F860203AB9DC6D2CB12046B9
:1012E00001F074F9204605F0FBF9BDE81040034811
:1012F00001F06CB9302300203C6A000878330020EC
:10130000014B1870704700BFF812002010B54FF065
:1013100000540C4B22689A4211D10B4B627D1A701B
:101320000A48237D03730A49C9220E3000F0BCFA33
:10133000E0220021204600F0DDFA012010BD00204F
:10134000FCE700BF9AAD44C5F8120020003400202D
:101350001600002037B501F0D1FB194D194928813D
:101360000223012218486B7100F07CFF00230193D7
:10137000164B174900931748174B4FF4805201F052
:101380007DFE164B197811B1124801F09DFE01F057
:101390009FFA0446FFF7F2FC4FF4C873B0FBF3F278
:1013A00002FB130304F5167010FA83F00C4B18605F
:1013B00004F050F808B10F232B8103B030BD00BFFB
:1013C000EC12002040420F0030230020ED0F0008F7
:1013D000FC1200200423002075100008F8120020E1
:1013E000002300202DE9F04F2DED028B0FF25C2938
:1013F000D9E900898B4C93B08B4E8C4F204601F07D
:1014000039FF034660B30025CDE90F550E95ADF8C1
:101410004450027B8DF8442099684068DFF834A27C
:101420000FAA03C21B6843F000430E9301F052FA67
:10143000821941F1000300950EA9384600F040FBE7
:10144000A84205DD204601F019FF8AF80050D5E7D3
:101450009AF80030072B00F2B58001338AF800308B
:101460000BAE9FED6C8B0023704FDFF8ECA10A935D
:10147000ADF834300B9373604FF0000B5B468DED8D
:10148000008B01250DF11D0207A938468DF81C506F
:101490008DF81DB000F096FE9DF81C30002B40F03A
:1014A0009580204601F018FE0646002845D1604F81
:1014B00001F00EFA3B6898423FD301F009FA8246E8
:1014C000FFF75CFC4FF4C8730AF5167AB0FBF3F231
:1014D00002FB13031AFA83F33B60564F97F800B0F0
:1014E000CBF1100ABBF1000F14BF33462B465FFA55
:1014F0008AFA0EA88DF82830FFF758FCBAF1060FCB
:1015000028BF4FF0060A0EAB03EB0B0152460DF15C
:10151000290000F0C9F90AAB0393182302930AF1DA
:101520000102454BD2B2CDE90053049220463BA3C1
:10153000D3E9002301F0D2FD3E7001F0C9F93F4A22
:101540003F4D1368C31AB3F57A7F2ED3106001F0B4
:10155000C1F902460B46204601F09AFE204601F0F2
:10156000BBFD10B32B7B374E002B14BF032302238C
:10157000737101F0ADF90EAF4FF47A730122B0FB35
:10158000F3F039463060304601F04EFA18230293EA
:101590002D4B019380B240F25513CDE903700093B7
:1015A00042464B46204601F099FD2B7B2BB1FFF7BD
:1015B00075FC2B7B002B7FF41FAF13B0BDEC028BAF
:1015C000BDE8F08F204601F059FE49E7DAF8143003
:1015D00083F08003CAF81430594610220EA800F098
:1015E00089F90DF11E0308AA0AA9384600F066FB26
:1015F00096E803000FAB83E803009DF834308DF8C4
:1016000044300A9B0E930EA9DDE90823204601F021
:10161000FDFF31E70000000000000000401DA12098
:1016200026812A0B0423002040420F003023002093
:1016300000230020FD220020FC220020E0340020B6
:1016400000340020EC120020E4340020F1C6A7C1D1
:10165000D068080FE53400200004004808B50548AC
:1016600000F0C6FBBDE80840034A0449002005F02D
:1016700031B800BF3023002038350020C9120008DF
:101680002DE9F84F4FF47A73DFF85880DFF858905F
:1016900006460D4602FB03F7002498F900305A1C59
:1016A0005FFA84FA01D0A34212D159F824000368EA
:1016B0002A46D3F820B031463B46D847854207D169
:1016C000074B012083F800A0BDE8F88F0124E4E770
:1016D000002CFBD04FF4FA7003F07CFA0020F3E703
:1016E0002C350020181100201C11002007B5002304
:1016F000024601210DF107008DF80730FFF7C0FF0A
:1017000020B19DF8070003B05DF804FB4FF0FF30F7
:10171000F9E700000A4608B50421FFF7B1FF80F0A1
:101720000100C0B2404208BD30B4074B0A461978E8
:10173000064B53F821402368DD69054B0146AC4652
:10174000204630BC604700BF2C3500201C11002013
:10175000A086010070B503F0D7FC094E094D30801A
:10176000002428683388834208D903F0C9FC2B6819
:1017700004440133B4F5204F2B60F2D370BD00BF99
:101780002E350020E834002003F07EBD00F100601B
:1017900000F520400068704700F10060920000F5FD
:1017A000204003F0F5BC0000054B1A68054B1B8870
:1017B0009B1A834202D9104403F0A2BC0020704758
:1017C000E83400202E35002038B5084D044629B1F4
:1017D00028682044BDE8384003F0AABC28682044AB
:1017E00003F094FC0028F3D038BD00BFE83400209B
:1017F0000020704700F10050A0F51040D0F890058F
:1018000070470000064991F8243033B10023086A7C
:1018100081F824300822FFF7BFBF0120704700BFC6
:10182000EC340020014B1868704700BF002004E032
:1018300070B50E4B5C6893F90860421E0A44013C87
:101840000B46934207D214F9015F581C2DB100F8E2
:10185000015C0346F5E7184605E02C2482421C7023
:1018600001D9981C5E70401A70BD00BF2411002081
:10187000022802BF014B80229A6170470004004891
:10188000022802BF024B4FF400029A61704700BF6A
:1018900000040048022801BF024A536983F0800314
:1018A000536170470004004810B50023934203D0F1
:1018B000CC5CC4540133F9E710BD000010B5013809
:1018C00010F9013F3BB191F900409C4203D11AB19C
:1018D0000131013AF4E71AB191F90020981A10BDCC
:1018E0001046FCE703460246D01A12F9011B0029F4
:1018F000FAD1704702440346934202D003F8011B19
:10190000FAE770472DE9F8431F4D144695F8242057
:101910000746884652BBDFF870909CB395F8243098
:101920002BB92022FF2148462F62FFF7E3FF95F8ED
:101930002400C0F10802A24228BF2246D6B2414686
:10194000920005EB8000FFF7AFFF95F82430A41B51
:101950001E44F6B2082E17449044E4B285F8246081
:10196000DBD1FFF74FFF0028D7D108E02B6A03EB4C
:1019700082038342CFD0FFF745FF0028CBD1002060
:10198000BDE8F8830120FBE7EC340020024B1A7815
:10199000024B1A70704700BF2C3500201811002030
:1019A00038B5194C194D204602F016FC2946204640
:1019B00002F03EFC2D681648EA6ED2F8043843F077
:1019C0000203C2F8043803F005F92846114902F071
:1019D00037FDEA6E104DD2F8043828680F4923F01D
:1019E0000203C2F80438A0424FF461430B6001D0F7
:1019F00002F052FB6868A04204D0BDE838400749B5
:101A000002F04ABB38BD00BF60370020946B00086D
:101A100040420F009C6B00081C1100201435002070
:101A200070B50C4B0C4D1E780C4B55F826209A4285
:101A300004460DD00A4B002118221846FFF75AFF22
:101A40000460014655F82600BDE8704002F024BB52
:101A500070BD00BF2C3500201C1100206037002015
:101A600014350020202383F3118862B670470000EC
:101A7000002383F3118862B67047000010B4026837
:101A800054681A4623465DF8044B184701207047F6
:101A9000002070470020704770470000002070470A
:101AA0000E20704700F5805090F8C800C0F3400049
:101AB0007047000000F5805090F9C90070470000A1
:101AC0002DE9F0410C68BDF8187014F000541E4662
:101AD0006FD10B7B082B6CD8FFF7C4FF4569AB684F
:101AE0005B010CD4AB681B0108D4AC6814F08054C3
:101AF0005DD1FFF7BDFF2046BDE8F08101240B68F2
:101B000004F1180C002BB8BFDB004FEA0C1CB4BF6B
:101B100043F004035B0545F80C300B680FFA84FCB6
:101B200013F0804F18BF05EB0C1E05EB0C1C1EBFFD
:101B3000DEF8803143F00203CEF880310B7BCCF825
:101B4000843105EB04158B68C5F88C314B68C5F8FA
:101B50008831DCF8803143F00103CCF8803100EBB0
:101B6000441541F268031D4403EB44130344C5E9E3
:101B7000002608330D4601F10C0C55F804EB43F830
:101B800004EB6545F9D184342D881D8000EB4414A5
:101B900007F00303257925F00B052B432371FFF78D
:101BA00067FF06973346BDE8F04100F0AFBC022462
:101BB000A5E74FF0FF309FE713B500F58054019182
:101BC000E06D00F039FD1F280AD90199E06D20224F
:101BD00000F0A8FDA0F120035842584102B010BD0A
:101BE0000020FBE708B500F58050FFF73BFFC06D14
:101BF00000F0F6FCBDE80840FFF73ABF00220260A3
:101C0000828142608260704710B500220023C0E9E3
:101C100000230023044603810C30FFF7EFFF20462A
:101C200010BD0000F0B5054600F580500C4690F858
:101C3000C83013F0040FC3F3800108BF114661F3ED
:101C4000820304F1840680F8C83005EB461389B09E
:101C50001B79D8072ED57AB319072DD46846FFF71C
:101C6000D3FF05EB441303F5835303F1180703AACD
:101C7000103318685968144603C40833BB4222461F
:101C8000F7D1186820609B88A380DDE90E23CDE999
:101C900000230123ADF808302B686946DB6B28462A
:101CA000984705EB46152B791A075CBF43F00803EC
:101CB0002B7101E0002AF4D109B0F0BD2DE9F04705
:101CC000074688B007F5805468469A468846FFF76D
:101CD000C9FE9146FFF798FFE06D00F093FC1F28C6
:101CE00029D9E06D2022694600F09EFD202822D1EE
:101CF00003AD444605AB2E4603CE9E422060616094
:101D0000354604F10804F6D130682060B388A3801A
:101D1000DDE90023C9E90023BDF80830AAF8003046
:101D2000FFF7A6FE4A4653464146384608B0BDE88E
:101D3000F04700F0D9BBFFF79BFE002008B0BDE8DC
:101D4000F08700002DE9F84F0023C0E90133254B4F
:101D5000044640F8183B0F46FFF750FF04F12800F7
:101D6000FFF752FF04F1480804F58255464608354E
:101D700030462036FFF748FFAE42F9D104F58055D2
:101D80004FF480534FF00009C5E91339C5F8488076
:101D90000123EE6504F5875804F58456C5F8549080
:101DA00085F8583085F86030083608F108084FF09B
:101DB000000A4FF0000B46E908ABA6F11800FFF748
:101DC0001DFF203646F8289C4645F4D185F8C97099
:101DD00017B1054800F076FD044B63612046BDE86D
:101DE000F88F00BF3C6A0008146A000800640040D5
:101DF00010B5044B197804464A1C1A70FFF7A2FF6D
:101E0000204610BD343500202DE9F047002950D080
:101E1000294B2A4FB7FBF1F599428CBF0A231123B6
:101E2000581EB5FBF3FC03FB1C53C4B22BB10228B4
:101E30000346F5D80020BDE8F0870CF1FF36B6F573
:101E4000806FF7D2C4EBC40E0EF103034FEAE3092F
:101E5000C3F3C703A4EB030809F1010A4FF47A7531
:101E60005FFA88F009FB05555AFA88F8B5FBF8F5D2
:101E7000B5F5617FC1BF0EF1FF33C3F3C703E01AAD
:101E8000C0B25C1C50FA84F40CFB04F4B7FBF4F40D
:101E9000A142CFD1013BDBB20F2BCBD80138C0B26E
:101EA0000728C7D80021107116809170D3700120C7
:101EB000C1E70846BFE700BF3F420F0000B4C404BB
:101EC00070B505460E464FF47A746B695B6803F093
:101ED0000103B34207D04FF47A7002F07BFE013C5D
:101EE000F3D1204670BD0120FCE7000030B5426907
:101EF000936913F0700F16D000230B4C936103F11C
:101F0000840200EB421211794D0709D5890707D5E4
:101F1000416954F823508D60117941F00401117129
:101F20000133032BEBD130BD286A000873B51D4681
:101F3000436916469A68D207044609D59A68012172
:101F40009960C2F34002CDE900650021FFF76AFE07
:101F500063699A68D1050BD59A684FF480719960CE
:101F6000C2F34022CDE9006501212046FFF75AFE69
:101F700063699A68D2030BD59A684FF480319960EF
:101F8000C2F34042CDE9006502212046FFF74AFE38
:101F9000204602B0BDE87040FFF7A8BFF8B5044680
:101FA000466900296CD106F10C07386880076AD0B1
:101FB00006EB01153868D5F8B00110F0040FD5F81C
:101FC000B0011ABFC00840F00040400DA061D5F834
:101FD000B0C11CF0020F1CBF40F08040A061D5F8DA
:101FE000B40106EB011100F00F0084F82400D1F8D1
:101FF000B8012077D1F8B801000A6077D1F8B801AC
:10200000000CA077D1F8B801000EE077D1F8BC0140
:1020100084F82000D1F8BC01000A84F82100D1F82E
:10202000BC01000C84F82200D1F8BC11090E84F820
:1020300023103821396004F1340004F1180104F14F
:10204000240551F8046B40F8046BA942F9D10988C2
:102050000180C4E90A2321460023238651F8283B46
:102060002046DB6B984704F58052204692F8C83032
:1020700043F0040382F8C830BDE8F840FFF736BFEC
:1020800006F1100791E7F8BD10B5044600F022FCF8
:1020900002460B4652EA030102D0013A63F1000303
:1020A0000449086820B12146BDE81040FFF776BF1B
:1020B00010BD00BF30350020F8B500F583511E4635
:1020C000FFF7D0FCDFF844C00831002404F1840598
:1020D00000EB45152B795F070ED4DB060CD5D1E953
:1020E00000739742B34107D243695CF824709F6044
:1020F0002B7943F004032B710134032C01F12001EF
:10210000E4D1BDE8F840FFF7B3BC00BF286A00087F
:1021100008B5FFF7A7FCFFF7E9FEBDE80840FFF7A9
:10212000A7BC0000F8B543690546986800F0E05088
:10213000B0F1E05F0F461FD0E8B1FFF793FC05F563
:1021400083541034002606F1840305EB43131B79F6
:102150001A0706D50136032E04F12004F3D101201D
:1021600007E05B07F6D42146384600F009FA00285C
:10217000F0D1FFF77DFCF8BD0120FCE700F58050B1
:1021800008B5FFF76FFCC06D00F03CFAFFF770FC7C
:1021900043090CBF0120002008BD0000F8B51D4612
:1021A000002313700F4606461446FFF7E7FF80F042
:1021B0000100387025B129463046FFF7B3FF207083
:1021C000F8BD00002DE9B8410C4615461F46804673
:1021D00000F080FB0B462178024609B9287850B1FF
:1021E0004046FFF769FFFFF793FF3B462A4621462B
:1021F000FFF7D4FF0120BDE8B881000010B5FFF75C
:1022000031FC174B9A6D42F000729A659A6B42F05E
:1022100000729A639A6B00F5805422F000729A6300
:10222000FFF726FC94F8C830DB0718D4B9B10221B7
:102230001320FFF717FC01F07DFD0221142001F0AF
:1022400079FD0221152001F075FD94F8C83043F0A6
:10225000010384F8C830BDE81040FFF709BC10BD89
:10226000001002402DE9F04700F5805588B095F840
:10227000C930012B0446884616467FD8804F57F850
:1022800023200AB947F82300D7F800A0C4F80C802F
:102290002674BAF1000F63D095F8C930012B6FD0C6
:1022A00001212046FFF7AAFFFFF7DCFB62691368F4
:1022B00023F0020313606269136843F001031360A3
:1022C000636900275F6101212046FFF7D1FBFFF71B
:1022D000F7FD002800F09580E86D00F081F904F525
:1022E0008359BA4609F10809202200216846FFF700
:1022F00001FB02A8FFF782FCCDF818A06A4609EBA3
:1023000007030DF1180E9446BCE80300F44518606D
:102310005960624603F10803F5D1DCF8000018604B
:1023200020379CF804201A71602FDDD195F8C83051
:102330006FF38203002785F8C8306A46414620467D
:10234000ADF80070ADF802708DF80470FFF75CFD19
:10235000636948BB4FF400421A6008B0BDE8F087DB
:1023600041F2D00004F0BEF9814610B15146FFF7AA
:10237000E9FCC7F80090B9F1000F8DD10020ECE71F
:10238000386803681B6B98470146002888D1386875
:10239000FFF734FF3868036832465B684146984768
:1023A00000287FF47DAFE9E761221A609DF80230D2
:1023B0009DF803201B06120402F4702203F0407300
:1023C0001343BDF80020C2F3090213439DF8042013
:1023D0001205022E02F4E0020CBF4FF00041002172
:1023E000134362690B43D361636913225A616269C3
:1023F000136823F00103136039462046FFF760FDA0
:1024000008B96369A6E795F8C93093BB6169D1F84B
:10241000002242F00102C1F800226169D1F80022D5
:1024200022F47C5222F00E02C1F800226169D1F838
:10243000002242F46062C1F800226269C2F81432DC
:102440006269C2F80432626941F6FF71C2F80C1287
:102450006269C2F840326269C2F84432636901229B
:10246000C3F81C226269D2F8003223F00103C2F8DB
:10247000003295F8C83043F0020385F8C8306CE7A5
:102480003035002008B500F025FA50EA0103024675
:1024900002D0421E61F10001044B186810B10B46D6
:1024A000FFF744FDBDE8084001F00EBB30350020C9
:1024B00008B50020FFF7E8FDBDE8084001F004BBC7
:1024C00008B50120FFF7E0FDBDE8084001F0FCBAC7
:1024D00013B56C4684E80600031D94E8030083E806
:1024E0000500012002B010BD73B58568019155B19A
:1024F0001B885B0707D4D0E900369B6B9847019A8D
:10250000C1B23046A847012002B070BDF0B5866860
:1025100089B005460C465EB1BDF838305B070AD479
:10252000D0E900379B6B98472246C1B23846B04786
:10253000012009B0F0BD00220023CDE900230023D3
:10254000ADF808300A4603AB01F10806106851687F
:102550001C4603C40832B2422346F7D110682060FB
:102560009288A28000F0B8F90423ADF808302B68F7
:10257000CDE90001DB6B694628469847D8E70000A3
:1025800030B503680968DD0FB5EBD17F23F06044F7
:1025900021F060424FEAD1700BD0002BB8BFA40CE1
:1025A0000029B8BF920C944202D034BF0120002011
:1025B00030BD944205D1C1F38070C3F38073834270
:1025C000F6D194422CBF00200120F1E710B5037C26
:1025D000044613B9006804F0BDF8204610BD0000A1
:1025E0000023BFF35B8FC360BFF35B8FBFF35B8FD1
:1025F0008360BFF35B8F7047BFF35B8F0068BFF3EF
:102600005B8F704770B505460C30FFF7F5FF05F19D
:10261000080604463046FFF7EFFFA04206D93046D1
:102620006D68FFF7E9FF2544281A70BD3046FFF7B3
:10263000E3FF201AF9E7000070B50546406898B13D
:1026400005F10800FFF7D8FF05F10C0604463046F7
:10265000FFF7D2FF8442304694BF6D680025FFF734
:10266000CBFF013C2C44201A70BD000038B50C464D
:102670000546FFF7C7FFA04210D305F10800FFF79A
:10268000BBFF04446868B4FBF0F100FB1144BFF3E6
:102690005B8F0120AC60BFF35B8F38BD0020FCE78F
:1026A0002DE9F041144607460D46FFF7C5FF844269
:1026B00028BF0446D4B1B84658F80C6B4046FFF723
:1026C0009BFF3044286040467E68FFF795FF331A31
:1026D0009C4203D86C600120BDE8F0816B60A41BB4
:1026E0003B68AB602044E8600220F5E72046F3E752
:1026F00038B50C460546FFF79FFFA04210D305F101
:102700000C00FFF779FF04446868B4FBF0F100FBAC
:102710001144BFF35B8F0120EC60BFF35B8F38BDCA
:102720000020FCE72DE9FF41884669460746FFF790
:10273000B7FF6C4606B204EBC6060025B44209D0CA
:102740006268206808EB0501FFF7AEF8636808349B
:102750001D44F3E729463846FFF7CAFF284604B070
:10276000BDE8F081F8B505460C300F46FFF744FF91
:1027700005F1080604463046FFF73EFFA04230460A
:1027800088BF6C68FFF738FF201A386020B13046E8
:102790002C68FFF731FF2044F8BD000073B51446E4
:1027A00006460D46FFF72EFF844228BF04460190DF
:1027B000DCB101A93046FFF7D5FF019B33B9326880
:1027C000C5E90233C5E9002401200CE09C4238BF72
:1027D00001942860019868608442F5D93368AB6041
:1027E000241AEC60022002B070BD2046FBE7000016
:1027F0002DE9FF410F466946FFF7D0FF6C4600B256
:1028000004EBC0050026AC4209D0D4F8048054F88B
:10281000081BB8194246FFF747F84644F3E730462D
:1028200004B0BDE8F081000038B50546FFF7E0FFD1
:10283000044601462846FFF719FF204638BD000030
:1028400000B59BB0EFF3098168226846FFF72CF8CA
:10285000EFF30583044B9A6BDA6A9A6A9A6A9A6A6A
:102860009A6A9A6A9B6AFEE700ED00E000B59BB0A9
:10287000EFF3098168226846FFF716F8EFF3058346
:10288000044B9A6B9A6A9A6A9A6A9A6A9A6A9B6ADB
:10289000FEE700BF00ED00E000B59BB0EFF309815B
:1028A00068226846FFF700F8EFF30583034B5A6B85
:1028B0009A6A9A6A9A6A9A6A9B6AFEE700ED00E051
:1028C000FEE700000FB408B5029802F013F9FEE726
:1028D00002F01ABD02F0F2BC02F0F0BC2DE9F047A4
:1028E0000D46044600219046284640F27912FFF733
:1028F00001F8234620220021284600F03FFE231D38
:1029000002222021284600F039FE631D03222221E5
:10291000284600F033FEA31D03222521284600F09F
:102920002DFE04F1080310222821284600F026FE7F
:1029300004F1100308223821284600F01FFE04F19C
:10294000110308224021284600F018FE04F112036A
:1029500008224821284600F011FE04F11403202229
:102960005021284600F00AFE04F11803402270218D
:10297000284600F003FE04F120030822B021284677
:1029800000F0FCFD04F121030822B821284600F0E4
:10299000F5FD04F12207C0263B46314608222846B1
:1029A000083600F0EBFDB6F5A07F07F10107F3D183
:1029B00004F1320308223146284600F0DFFD0027EB
:1029C00004F1330A94F832304FEAC7099F4209F5FF
:1029D000A47615D3B8F1000F08D1314604F59973E8
:1029E0000722284600F0CAFD09F24F16274694F840
:1029F00032213B1B93420CD3F01DC008BDE8F08789
:102A00000AEB070308223146284600F0B7FD0137DC
:102A1000D8E707F2331331460822284600F0AEFD0E
:102A200008360137E3E7000013B5044608460021E5
:102A300001602346C0F803102022019000F09EFDA3
:102A40000198231D0222202100F098FD0198631DAA
:102A50000322222100F092FD0198A31D03222521CB
:102A600000F08CFD019804F108031022282100F0E9
:102A700085FD072002B010BDF8B50E460546144688
:102A8000002181223046FEF735FF2B460822002127
:102A9000304600F073FD7CB96B1C072208213046DC
:102AA00000F06CFD0F2401236A785F1C013B934208
:102AB00004D3E01DC008F8BD0824F4E7EB19214653
:102AC0000822304600F05AFD08343B46ECE700008F
:102AD00030B5094D0A4491420DD011F8013B5840E0
:102AE000082340F30004013B2C4013F0FF0384EA69
:102AF0005000F6D1EFE730BD2083B8ED73B5384A0A
:102B0000106851686B4603C36A4636493648082345
:102B100003F038FE044670B9344A106851686B46B9
:102B200003C36A4632493048082303F02BFE0446AB
:102B300030BB0A2022E00369B3F5583FECD8418B43
:102B400040F217429142E7D12A4A024402F11001B1
:102B50008B42E1D3103B244900209D1AFFF7B8FFB8
:102B60002A46064604F118010020FFF7B1FFA368CA
:102B70009E42D1D1E3689842CED1002002B070BD10
:102B80000369B3F5583F22D8B0F8661040F21742F7
:102B900091421ED1174A024402F15C018B421AD3C2
:102BA0005C3B114900209D1AFFF792FF2A4606461A
:102BB00004F164010020FFF78BFFA26896420346F0
:102BC0000BD1E068834214BF0D200020D6E70B2014
:102BD000D4E70C20D2E71020D0E70D20CEE700BFCD
:102BE0007C6A0008DC5F030000A00008856A00081A
:102BF000905F03000860FFF72DE9F041C56915B942
:102C0000C161BDE8F0814B6823F06047C3F38A4699
:102C10004FEAD37EC3F3807816EA230638BF3E46D8
:102C2000AC462B465A68BEEBD27F22F060440AD0F5
:102C3000002A18DAA40CB44217D19D420FD10D60BE
:102C4000DEE71346EEE7A74207D102F08044C2F365
:102C5000807242450BD054B1EFE708D2EDE7CCF8D3
:102C600000100B60CDE7B44201D0B442E5D81A6839
:102C70009C46002AE5D11960C3E700002DE9F04722
:102C8000089D01F007044FEAD508224405F0070526
:102C900000EBD1004FF47F49944201D1BDE8F087A9
:102CA00004F0070705F0070A57453E4638BF564669
:102CB000C6F10806111B8E4228BF0E46E10808EB3C
:102CC000D50E415C13F80EC0B94029FA06F721FA77
:102CD0000AF1FFB28CEA010147FA0AF739408CEA9F
:102CE000010C03F80EC034443544D5E780EA0120D6
:102CF000082341F2210201B24000002980B203F111
:102D0000FF33B8BF504013F0FF03F4D17047000009
:102D100038B50C468D18A54200D138BD14F8011BFA
:102D2000FFF7E4FFF7E7000002684AB113680360A9
:102D3000C388018901339BB29942C38038BF0381A4
:102D40001046704770B588B0202204460D4668468C
:102D50000021FEF7CFFD20460495FFF7E5FF024670
:102D600058B16B46054608AE1C4603CCB4422860F9
:102D70006960234605F10805F6D1104608B070BD1C
:102D8000082817D909280CD00A280CD00B280CD0F9
:102D90000C280CD00D280CD00E2814BF4020302059
:102DA00070470C207047102070471420704718207F
:102DB0007047202070470000082817D90C280CD92C
:102DC00010280CD914280CD918280CD920280CD973
:102DD00030288CBF0F200E207047092070470A2032
:102DE00070470B2070470C2070470D207047000083
:102DF00010B54B6823B9CA8A63F30902CA8210BDB1
:102E0000C4681A681C60C360438A013B43824A60FD
:102E1000EFE700002DE9F84F1D46CB8A0F46C3F3BC
:102E200009010529814692460B4630D00020AAB2FE
:102E300007F11A049EB2042E1FFA80F80FD89045AD
:102E400003F1010306D3FB8A0A4462F30903FB8200
:102E500001201AE01AF80060E6540130EAE79045D4
:102E6000F1D2A1F1050B1C237C68BBFBF3F203FB41
:102E700012BB1FFA8BF6002C45D14846FFF754FFD2
:102E8000044638B978606FF00200BDE8F88F4FF063
:102E90000008E6E7002606607860ADB24FF0000B50
:102EA000454510D90AEB0803221D13F8011B915563
:102EB000B1B208F101081B291FFA88F82BD045454B
:102EC00006F10106F1D8FB8AC3F30902154465F344
:102ED0000903BCE7013292B21C462368002BF9D1EA
:102EE0006B1F0B441C21B3FBF1F301339BB29A42DD
:102EF000D3D2BBF1000FD0D14846FFF715FF20B960
:102F0000C4F800B0BFE70122E7E7C0F800B05E46B2
:102F100020600446C1E74545D5D94846FFF704FF80
:102F200008B92060AFE7C0F800B000262060044672
:102F3000B6E700002DE9F04F2DED028B83B0CDE90F
:102F40000013BDF83C5007469146002A00F09280DD
:102F50002DB10E9B002B00F08D80072D32D807F18C
:102F60000C00FFF7E1FE044638B96FF0020420467A
:102F700003B0BDEC028BBDE8F08F14220021FEF7F8
:102F8000B9FC0E992A4604F10800FEF78DFC681C76
:102F9000C0B2FFF711FFFFF7F3FE207499F800307D
:102FA000013814FA80F003F01F0363F03F0303724B
:102FB000009B43F00041616038462146FFF71CFE4C
:102FC0000124D4E700F10C034FF0000808EE103A9A
:102FD0004FF0800A4646444618EE100AFFF7A4FE5A
:102FE00083460028C1D014220021FEF783FCC6BB13
:102FF000019BABF8083002200E9B00F108029919E2
:103000005BFA82F20130C0B2082801D0AE422AD366
:10301000FFF7D2FEFFF7B4FE99F80020009B411E97
:1030200002F01F0242EA4812AE4208BF4FF0400AC7
:103030005BFA81F14AEA020A43F0004281F808A0F3
:103040008BF81000CBF8042059463846FFF7D4FD22
:103050000134AE4224B288F001084FF0000ABBD11F
:1030600085E70020C8E711F801CB02F801CB013653
:10307000B6B2C7E76FF0010479E70000F8B515466E
:103080000E462822002104461F46FEF733FC069B0D
:103090006360B5F5001F079BA76034BF6A094FF650
:1030A000FF72236204F10C0097B200239A4205D804
:1030B0000023036027826382A382F8BD0660013388
:1030C00030462036F2E7000003781BB94BB2002BE4
:1030D000C8BF017070470000007870472DE9F74FB6
:1030E000DDF83C90BDF830500D9E9DF83840BDF89D
:1030F0004070804692469B46B9F1000F01D1002FE7
:1031000051D11F2C4FD898F80000B0B9072F47D8DD
:1031100035F0030347D13A4649464FF6FF70FFF7B3
:10312000F7FD20F001002D02400445EA0464400C44
:1031300044EA40244FF6FF7321E040EA0520072FC0
:1031400040EA0464F6D900254FF6FF73C5F120006C
:10315000A5F120022AFA05F10BFA00F001432BFA3F
:1031600002F211431846C9B2FFF7C0FD0835402DE1
:103170000346EBD13A464946FFF7CAFD0346CDE97F
:103180000097324621464046FFF7D4FE337801339C
:10319000DBB21F2B88BF0023337003B0BDE8F08F74
:1031A0006FF00300F9E76FF00100F6E72DE9F04F4B
:1031B00085B09246DDF848800F9D9DF840209DF82F
:1031C0004490BDF84C7006469B46B8F1000F01D103
:1031D000002F48D11F2A46D83378002B46D00C0246
:1031E00044EA02649DF8381044EAC93444EA0144D0
:1031F0001C43072F44F0800432D900234FF6FF729E
:10320000C3F1200CA3F120002AFA03F10BFA0CFC05
:1032100041EA0C012BFA00F00143C9B210460393B6
:10322000FFF764FD039B0833402B0246E8D13A4682
:103230004146FFF76DFD0346CDE900872A4621464A
:103240003046FFF777FEB9F1010F06D12B78013335
:10325000DBB21F2B88BF00232B7005B0BDE8F08FB9
:103260004FF6FF73E8E76FF00100F6E76FF0030039
:10327000F3E70000C06900B104307047C3691A6801
:10328000C261C2681A60C360438A013B43827047CF
:103290002DE9F041D0F81880194E14461D464146DC
:1032A000002709B9BDE8F081D1E90223A21A65EB34
:1032B0000303964277EB03031ED283698B420DD141
:1032C000FFF796FD83691B688361C3680B60438ABF
:1032D000C1608169013B43828846E2E7FFF788FDD0
:1032E0000B68C8F80030C3680B60438AC160013BBB
:1032F0004382D8F80010D4E788460968D1E700BFB8
:1033000080841E002DE9F04F8BB00D46DDF8509003
:1033100014469B468046002800F01981B9F1000F41
:1033200000F01581531E3F2B00F21181012A03D1B9
:10333000BBF1000F40F00B810023CDE90833B8F852
:103340001430B5EBC30F4FEAC30703D300200BB013
:10335000BDE8F08F2B199F42D8F80C303ABF7F1B85
:10336000FFB227461BB9D8F81030002B7AD0272D92
:103370004ED8C5F12806B7424FF000032CBFF6B275
:103380003E4600932946D8F8080008AB3246FFF7BE
:1033900075FCA7EB060A35445FFA8AFAB8F81430D0
:1033A00003F10053053BDB000493D8F80C30039382
:1033B0002821039B13B1BAF1000F2CD1D8F81000CB
:1033C00040B1BAF1000F05D0009608AB5246691A19
:1033D000FFF754FC38B2002FB8D066070AD00AAB0A
:1033E00003EBD401624211F8083C02F007021341DA
:1033F00001F8083C082C3CD9102C40F2B580202C58
:1034000040F2B780BBF1000F00F09C80082334E04D
:10341000BA460026C2E7049BE02B28BFE0230693B0
:103420000B44AB42059314D95A1B0398009692455E
:1034300034BF5246D2B2691A08AB04300792FFF784
:103440001DFC079A1644AAEB020A1544F6B25FFA6D
:103450008AFA049B069A05999B1A0493039B1B689E
:103460000393A6E70093D8F8080008AB3A4629462C
:10347000AEE7BBF1000F13D00123B4EBC30F6CD048
:10348000082C12D89DF82030621E23FA02F2D507CC
:1034900006D54FF0FF3202FA04F423438DF82030B2
:1034A0009DF8203089F8003051E7102C12D8BDF873
:1034B0002030621E23FA02F2D10706D54FF0FF3208
:1034C00002FA04F42343ADF82030BDF82030A9F807
:1034D00000303CE7202C0FD80899631E21FA03F333
:1034E000DA0705D54FF0FF3202FA04F40C430894D2
:1034F000089BC9F800302AE7402C2BD0DDE908658D
:10350000611EC4F12102A4F1210326FA01F105FA9A
:1035100002F225FA03F311431943CB0712D5012216
:10352000A4F12003C4F1200102FA03F322FA01F10D
:10353000A240524243EA010363EB430332432B436D
:10354000CDE90823DDE90823C9E90023FFE66FF090
:103550000100FCE66FF00800F9E6082CA0D9102C59
:10356000B3D9202CEED8C3E7BBF1000FADD00223B6
:1035700083E7BBF1000FBBD004237EE730B5012AFF
:10358000144638BF0124402C85B028BF40240025B4
:10359000012ACDE9025518D81B788DF80830630749
:1035A0000AD004AB03EBD405624215F8083C02F0E4
:1035B0000702934005F8083C00910346224600218B
:1035C00002A8FFF75BFB05B030BD082AE4D9102A3A
:1035D00003D81B88ADF80830E1E7202A8DBFD3E976
:1035E00000231B680293CDE90223D8E710B5CB680E
:1035F0001BB98B600B618B8210BDC4681A681C609C
:10360000C360438A013B4382CA60F0E72DE9F04F73
:1036100095B0CDE904230B6804460D461806C3F3A4
:10362000C01147BFC3F3C03BC3F306264FF0020BE4
:103630000E46002B80F2018213F0C04940F0FD815C
:103640002A7B002A00F0F981BBF1020F03D0207819
:10365000B04240F0F581C3F30460089003F07F00AE
:10366000069059B3C3F3074A2A44069B92F8038095
:10367000760646EA0B4646EA834600220023CDE959
:103680000A235FEAD81346EA0A0603936AD0069B28
:10369000009367685B4652460AA92046B84700284F
:1036A00000F0D181A76987B9314604F10C00FFF71A
:1036B00049FB0746C8B96FF0020057E0C3F30F2A71
:1036C000590608BF0AF0030ACEE73B699E420DD0B7
:1036D0003F68002FF9D1314604F10C00FFF732FBAF
:1036E00007460028E7D0A3693B60A761FE7D08F08C
:1036F0001F03C6F38406F01A1FFA80FC0028B8BF27
:103700000CF120000793A3EB06031FFA83FCD7E913
:103710000221B8BF00B2002B0993BEBF0CF12003F9
:103720001BB2099352EA010335D0049EDFF8D4C2DC
:10373000B21A059E66EB01010026944576EB010363
:1037400029D395F80DE097F81AC0E64516D1039BEA
:10375000002B78D001281EDCA948904276EB0103AB
:1037600016D338E0A76927B96FF00C0015B0BDE893
:10377000F08F3B699E42B9D03F68F4E7A048904281
:1037800076EB010301D30020F0E7039B002BFAD076
:10379000099B0F2B18DCFA7D4FEA880302F0030225
:1037A00003F07C031343FB7539462046FFF720FBEB
:1037B0006B7BBB76039B3BB9FB7DC3F38402013279
:1037C00062F38603FB75CFE76A7BBB7E9A42DAD150
:1037D000039B002B37D04FEA9813022B33D0049B66
:1037E000BB60059BFB60142200210FA8FEF782F846
:1037F000049B0C93059B0D932B1D0E932B7BADF817
:1038000046A0013BDBB2ADF84430079B8DF8493050
:10381000089B8DF84A30069B8DF84B3094F8243085
:103820008DF848B083F001038DF84C300CA9A368E3
:1038300020469847FB7DC3F38403013303F01F0345
:103840009B02FB829FE7FB7DC8F34012B2EBD31FC4
:1038500040F0FC80079AC3F38403934240F0F98060
:1038600003992B7B4FEA981200294DD0D2075DD4E3
:10387000032B40F2F180049BBB60059BFB602B7B1C
:10388000AE1D033BDBB23246394604F10C00FFF7B4
:10389000C1FA00280CDA39462046FFF7A9FAFB7D69
:1038A000C3F38403013303F01F039B02FB8202E78F
:1038B000DDE90A84AB883B834FF6FF73C9F1200032
:1038C000A9F1200228FA09F104FA00F0014324FAD0
:1038D00002F211431846C9B2FFF708FA09F10809C4
:1038E000B9F1400F0346E9D1B8822A7B033AD2B23C
:1038F0003146FFF70DFAFB7DB882DA43C2F3C012FE
:1039000062F3C713FB753EE782B92E1D013BDBB2A4
:103910003246394604F10C00FFF77CFA0028BADB86
:103920002A7BB88A013AD2B23146E2E7F98AC1F37A
:103930000901013B0429DAB25CD8281D002307F1F4
:103940001B069A4208D910F801CB06F801C00131D4
:1039500001330529DBB2F4D104990C9105990D913D
:10396000934207F11B010E9138BF043379680F9120
:1039700034BF55FA83F300231093FB8AADF846A0B9
:10398000C3F309031A44079B8DF84930089B8DF84F
:103990004A30069B8DF84B3094F82430ADF8442023
:1039A00083F001038DF84C3000238DF848B07B6024
:1039B0002A7BB88A013A291DFFF7AAF93B8BB88206
:1039C000834203D1A3680CA92046984720460CA93E
:1039D000FFF70CFEFB7DBA8AC3F38403013303F0C7
:1039E0001F039B02FB823B8B9A420CBF00206FF0AF
:1039F0001000BBE67B68002BAED0052006E000BFC0
:103A000040420F0080841E001C3033461E68002E8A
:103A1000FAD1091A081D2E1D184401EB090CBCF13E
:103A20001B0F5FFA89F397D89A4295D916F8013B94
:103A300000F8013B09F10109EFE76FF0090095E695
:103A40006FF00A0092E66FF00B008FE66FF00D004A
:103A50008CE66FF00E0089E66FF00F0086E600BF7F
:103A6000EFF3098305494A6B22F001024A63683388
:103A700083F30988002383F31188704700EF00E087
:103A8000202080F3118862B60C4B0D4AD96821F4CE
:103A9000E0610904090C0A43DA60D3F8FC20094903
:103AA00042F08072C3F8FC200A6842F001020A600A
:103AB0001022DA7783F82200704700BF00ED00E0A3
:103AC0000003FA05001000E010B5202383F31188ED
:103AD0000E4B5B6813F4006314D0F1EE103AEFF371
:103AE0000984683C4FF08073E361094BDB6B23660C
:103AF00084F3098800F0B0FF10B1064BA36110BD3C
:103B0000054BFBE783F31188F9E700BF00ED00E008
:103B100000EF00E02B0600082E060008026843684C
:103B20001143016003B1184770470000024A13684F
:103B300043F0C003136070470038014013B50D4CCB
:103B4000204600F09DFA04F114000B490094002374
:103B5000202200F05FF9094B09490094202204F16A
:103B6000380000F0D9F9074A074BC4E9172302B01F
:103B700010BD00BF3C350020A83500202D3B0008BB
:103B8000C83500200038014000B4C40430B5037CBF
:103B9000234C002918BF0C46012B0FD1214B984212
:103BA0000CD1214B1A6E42F480421A66D3F8802061
:103BB00042F48042C3F88020D3F880302268036E3C
:103BC000C16D846603EB5203B3FBF2F36268150424
:103BD00042BF23F0070503F0070343EA4503CB6028
:103BE000A36843F040034B60E36843F001038B603C
:103BF00042F4967343F001030B604FF0FF330B6206
:103C0000510505D512F0102205D0B2F1805F04D025
:103C100080F8643030BD7F23FAE73F23F8E700BF28
:103C2000906A00083C350020001002402DE9F04762
:103C3000C66D3768F46934622107054618D014F060
:103C4000080118BF8021E20748BF41F02001A30707
:103C500048BF41F04001600748BF41F48071202314
:103C600083F31188281DFFF759FF002383F3118880
:103C7000E2050AD5202383F311884FF40071281D33
:103C8000FFF74CFF002383F311884FF020094FF01A
:103C9000000A14F0200838D13B0616D54FF0200951
:103CA00005F1380A200610D589F31188504600F036
:103CB00067F9002836DA0821281DFFF72FFF27F0C3
:103CC00080033360002383F31188790614D56206DC
:103CD00012D5202383F31188D5E913239A4208D102
:103CE0002B6C33B11021281D27F04007FFF716FF7A
:103CF0003760002383F31188E30619D5AA6E136990
:103D0000B3B1BDE8F0475069184789F31188B38C07
:103D100095F864102846194000F0CCF98AF3118810
:103D2000F469B6E780B2308588F31188F469B9E7A1
:103D3000BDE8F08700F1604303F561430901C9B2B2
:103D400083F80013012200F01F039A4043099B00EF
:103D500003F1604303F56143C3F880211A607047A3
:103D6000F8B5154682680669AA420B46816938BFD4
:103D70008568761AB54204460BD218462A46FDF7E6
:103D800093FDA3692B44A361A3685B1BA360284632
:103D9000F8BD0CD918463246FDF786FDAF1BE16829
:103DA0003A463044FDF780FDE3683B44EBE71846B4
:103DB0002A46FDF779FDE368E5E700008368934252
:103DC000F7B51546044638BF8568D0E90460361A51
:103DD000B5420BD22A46FDF767FD63692B44636148
:103DE000A36828465B1BA36003B0F0BD0DD9324623
:103DF0000191FDF759FD0199E068AF1B3A46314446
:103E0000FDF752FDE3683B44E9E72A46FDF74CFD28
:103E1000E368E4E710B50A440024C361029B8460B0
:103E2000C0E90000C0E90511C1600261036210BD74
:103E300008B5D0E90532934201D1826882B982681F
:103E4000013282605A1C42611970D0E904329A42F0
:103E500024BFC3684361002100F0D8FE002008BDE4
:103E60004FF0FF30FBE7000070B5202304460E46FC
:103E700083F31188A568A5B1A368A269013BA3607B
:103E8000531CA36115782269934224BFE368A361A0
:103E9000E3690BB120469847002383F31188284635
:103EA00007E03146204600F0A1FE0028E2DA85F363
:103EB000118870BD2DE9F74F04460E461746984607
:103EC000D0F81C904FF0200A8AF311884FF0000BB5
:103ED000154665B12A4631462046FFF741FF0346A5
:103EE00060B94146204600F081FE0028F1D0002351
:103EF00083F31188781B03B0BDE8F08FB9F1000F90
:103F000003D001902046C847019B8BF31188ED1A1E
:103F10001E448AF31188DCE7C0E90511C160C36162
:103F20001144009B8260C0E9000001610362704798
:103F3000F8B504460D461646202383F31188A7687A
:103F4000A7B1A368013BA36063695A1C62611D703D
:103F5000D4E904329A4224BFE3686361E3690BB198
:103F600020469847002080F3118807E0314620461C
:103F700000F03CFE0028E2DA87F31188F8BD00006B
:103F8000D0E905239A4210B501D182687AB98268D6
:103F9000013282605A1C82611C7803699A4224BFF4
:103FA000C3688361002100F031FE204610BD4FF050
:103FB000FF30FBE72DE9F74F04460E4617469846BB
:103FC000D0F81C904FF0200A8AF311884FF0000BB4
:103FD000154665B12A4631462046FFF7EFFE0346F7
:103FE00060B94146204600F001FE0028F1D00023D0
:103FF00083F31188781B03B0BDE8F08FB9F1000F8F
:1040000003D001902046C847019B8BF31188ED1A1D
:104010001E448AF31188DCE702684368114301609B
:1040200003B11847704700001430FFF743BF00008A
:104030004FF0FF331430FFF73DBF00003830FFF77B
:10404000B9BF00004FF0FF333830FFF7B3BF0000B7
:104050001430FFF709BF00004FF0FF311430FFF7B5
:1040600003BF00003830FFF763BF00004FF0FF329E
:104070003830FFF75DBF000000207047FFF75EBDDE
:10408000044B03600023C0E902334360012303743F
:10409000704700BFA86A000810B52023044683F3C8
:1040A0001188FFF773FD02232374002383F3118823
:1040B00010BD000038B5C36904460D461BB9042184
:1040C0000844FFF7A9FF294604F11400FFF7B0FEEA
:1040D000002806DA201D4FF48061BDE83840FFF764
:1040E0009BBF38BD026843681143016003B11847A4
:1040F0007047000013B5446BD4F894341A681178F3
:10410000042915D1217C022912D1197912890123A0
:104110008B4013420CD101A904F14C0001F04EFF79
:10412000D4F89444019B21790246206800F0D4F928
:1041300002B010BD143001F0D1BE00004FF0FF33CB
:10414000143001F0CBBE00004C3001F0A3BF0000E2
:104150004FF0FF334C3001F09DBF0000143001F0F0
:104160009FBE00004FF0FF31143001F099BE0000F7
:104170004C3001F06FBF00004FF0FF324C3001F0C7
:1041800069BF00000020704710B5D0F894341A6859
:1041900011780429044617D1017C022914D15979D8
:1041A000528901238B4013420ED1143001F032FEAC
:1041B000024648B1D4F894444FF480736179206882
:1041C000BDE8104000F076B910BD0000406BFFF76D
:1041D000DBBF0000704700007FB5124B0360002377
:1041E0004360C0E90233012502260F4B05740446E3
:1041F0000290019300F18402294600964FF48073E7
:10420000143001F0E3FD094B0294CDE9006304F59D
:1042100023724FF48073294604F14C0001F0AAFE8A
:1042200004B070BDD06A0008CD410008F540000818
:104230000B68202282F311880A7903EB8202106254
:104240004A790D3243F822008A7912B103EB8203D6
:10425000186202230374C0F89414002383F31188B6
:104260007047000038B5037F044613B190F854300E
:10427000ABB9201D01250221FFF734FF04F1140022
:1042800025776FF0010100F0CDFC84F8545004F163
:104290004C006FF00101BDE8384000F0C3BC38BDF0
:1042A00010B5012104460430FFF71CFF00232377DB
:1042B00084F8543010BD000038B504460025143091
:1042C00001F09CFD04F14C00257701F06BFE201DF0
:1042D00084F854500121FFF705FF2046BDE838401F
:1042E000FFF752BF90F85C3003F06003202B07D13A
:1042F00090F85D20212A4FF0000303D81F2A06D82A
:1043000000207047222AFBD1C0E9143303E0034A9E
:104310000265072242658365012070473011002045
:1043200037B5D0F894341A681178042904461AD1A4
:10433000017C022917D11979128901238B4013427C
:1043400011D100F14C05284601F0ECFE58B101A94D
:10435000284601F033FED4F89444019B21790246AB
:10436000206800F0B9F803B030BD0000F0B500EBF4
:10437000810385B01E6A04460D46FEB1202383F3F7
:10438000118804EB8507301D0821FFF7ABFEFB68A1
:104390005B691B6806F14C001BB1019001F01CFE2B
:1043A000019803A901F00AFE024648B1039B294681
:1043B000204600F091F8002383F3118805B0F0BD8A
:1043C000FB685A691268002AF5D01B8A013B13402A
:1043D000F1D104F15C02EAE70D3138B550F8214023
:1043E000DCB1202383F31188D4F894241368527924
:1043F00003EB8203DB689B695D6845B104216018AB
:10440000FFF770FE294604F1140001F00DFD20466F
:10441000FFF7BAFE002383F3118838BD7047000010
:1044200001F0BAB810B501230446282200F8243B55
:104430000021FDF75FFA0023C4E9013310BD00003D
:1044400038B50446202383F311880025C0E90355BD
:10445000C0E90555C0E90755416001F0ADF80223F8
:10446000237085F3118838BD70B500EB81030546D4
:104470005069DA600E46144618B110220021FDF78B
:1044800039FAA06918B110220021FDF733FA31463C
:104490002846BDE8704001F059B90000826802F07A
:1044A000011282600022C0E90422C0E906220262F1
:1044B00001F0D8B9F0B400EB81044789E468012524
:1044C000A4698D403D43458123600023A260636061
:1044D000F0BC01F0F3B90000F0B400EB81040789EF
:1044E000E468012564698D403D4305812360002314
:1044F000A2606360F0BC01F06DBA000070B50223E9
:10450000002504460370C0E90255C0E90455C0E91E
:1045100006554566056280F84C5001F0B3F86368B3
:104520001B6823B129462046BDE87040184770BD7E
:10453000037880F868300523037043681B6810B562
:1045400004460BB1042198470023A36010BD00006E
:1045500090F86820436802701B680BB1052118476A
:104560007047000070B590F84C30044613B100233A
:1045700080F84C3004F15C02204601F095F9636844
:104580009B68B3B994F85C3013F0600535D0002116
:10459000204601F0FDFB0021204601F0EFFB63689F
:1045A0001B6813B1062120469847062384F84C3037
:1045B00070BD204698470028E4D0B4F86230626DA0
:1045C0009A4288BF636594F95C30656D002B4FF0AB
:1045D000200380F20381002D00F0F280092284F88C
:1045E0004C2083F311880021D4E914232046FFF7DF
:1045F00073FF002383F31188DAE794F85D2003F05A
:104600007F0343EA022340F20232934200F0C58066
:1046100021D8B3F5807F48D00DD8012B3FD0022B95
:1046200000F09380002BB2D104F1640222650222D3
:104630006265A365C1E7B3F5817F00F09B80B3F5A8
:10464000407FA4D194F85E30012BA0D1B4F864303F
:1046500043F0020332E0B3F5006F4DD017D8B3F545
:10466000A06F31D0A3F5C063012B90D8636894F894
:104670005E205E6894F85F10B4F860302046B04762
:10468000002884D043682365036863651AE0B3F5A6
:10469000106F36D040F6024293427FF478AF5C4B05
:1046A0002365022363650023C3E794F85E30012B82
:1046B0007FF46DAFB4F8643023F00203C4E91455FD
:1046C000A4F86430A56578E7B4F85C30B3F5A06F62
:1046D0000ED194F85E3084F86630204601F02AF856
:1046E00063681B6813B10121204698470323237098
:1046F0000023C4E914339CE704F167032365012315
:10470000C3E72378042B10D1202383F3118820469C
:10471000FFF7C4FE85F311880321636884F86750AE
:1047200021701B680BB12046984794F85E30002B2F
:10473000DED084F867300423237063681B68002B85
:10474000D6D0022120469847D2E794F860301D0663
:1047500003F00F0120460AD501F098F8012804D093
:1047600002287FF414AF2B4B9AE72B4B98E701F00C
:104770007FF8F3E794F85E30002B7FF408AF94F8ED
:10478000603013F00F01B3D01A06204602D501F0B5
:1047900013FBADE701F006FBAAE794F85E30002BAF
:1047A0007FF4F5AE94F8603013F00F01A0D01B0633
:1047B000204602D501F0ECFA9AE701F0DFFA97E71C
:1047C000142284F84C2083F311882B462A4629466C
:1047D0002046FFF76FFE85F31188E9E65DB11522EB
:1047E00084F84C2083F311880021D4E91423204657
:1047F000FFF760FEFDE60B2284F84C2083F311885E
:104800002B462A4629462046FFF766FEE3E700BF0F
:10481000006B0008F86A0008FC6A000838B590F8D8
:104820004C300446002B3ED0063BDAB20F2A34D877
:104830000F2B32D8DFE803F0373131082232313123
:104840003131313131313737456DB0F862309D4209
:1048500014D2C3681B8AB5FBF3F203FB12556DB982
:10486000202383F311882B462A462946FFF734FE7E
:1048700085F311880A2384F84C300EE0142384F861
:104880004C30202383F3118800231A461946204612
:10489000FFF710FE002383F3118838BD836D03B149
:1048A00098470023E7E70021204601F071FA002134
:1048B000204601F063FA63681B6813B106212046A5
:1048C00098470623D7E7000010B590F84C30142B1A
:1048D000044629D017D8062B05D001D81BB110BD2E
:1048E000093B022BFBD80021204601F051FA0021A0
:1048F000204601F043FA63681B6813B10621204685
:104900009847062319E0152BE9D10B2380F84C308A
:10491000202383F3118800231A461946FFF7DCFD94
:10492000002383F31188DAE7C3689B695B68002B77
:10493000D5D1836D03B19847002384F84C30CEE77E
:10494000024B0022C3E900339A607047E83500202B
:10495000002303748268054B1B6899689142FBD25F
:104960005A6803604260106058607047E835002064
:1049700008B5202383F31188037C032B05D0042B77
:104980000DD02BB983F3118808BD436900221A604A
:104990004FF0FF334361FFF7DBFF0023F2E7D0E97D
:1049A000003213605A60F3E7002303748268054BFA
:1049B0001B6899689142FBD85A6803604260106096
:1049C00058607047E8350020054B1969087418686D
:1049D00002681A605360186101230374FBF710BE6C
:1049E000E835002030B54B1C0B4D87B0044610D085
:1049F0002B690A4A01A800F031F92046FFF7E4FFCD
:104A0000049B13B101A800F065F92B69586907B040
:104A100030BDFFF7D9FFF8E7E835002071490008FD
:104A200038B50C4D41612B6981689A689142044602
:104A300003D8BDE83840FFF78BBF1846FFF7B4FF37
:104A400001232C61014623742046BDE83840FBF762
:104A5000D7BD00BFE8350020044B1A681B69906879
:104A60009B68984294BF002001207047E8350020E1
:104A700010B5084C236820691A682260546001222E
:104A800023611A74FFF790FF01462069BDE81040CA
:104A9000FBF7B6BDE835002008B5FFF7DDFF18B11C
:104AA000BDE80840FFF7E4BF08BD0000FFF7E0BF26
:104AB000FEE7000010B50C4CFFF742FF00F0C0F815
:104AC0000A498022204600F047F8012344F8180CD8
:104AD0000374FEF7D5FF002383F3118862B6044800
:104AE000BDE8104000F058B810360020046B0008F4
:104AF000146B000808B572B6034B586200F0D8FB7F
:104B000000F084FCFEE700BFE835002000F01CB98F
:104B1000EFF3118020B9EFF30583202282F311888F
:104B20007047000010B530B9EFF30584C4F30804F2
:104B300014B180F3118810BDFFF7AEFF84F3118824
:104B4000F9E70000034A516853685B1A9842FBD8A2
:104B5000704700BF001000E08260022202827047AE
:104B60008368A3F17C0243F80C2C026943F83C2CC7
:104B7000426943F8382C074A43F81C2CC26843F8B2
:104B8000102C022203F8082C002203F8072CA3F1B2
:104B9000180070471906000810B5202383F3118808
:104BA000FFF7DEFF00210446FFF73AFF002383F3FF
:104BB0001188204610BD0000024B1B6958610F2070
:104BC000FFF702BFE8350020202383F31188FFF7A9
:104BD000F3BF000008B50146202383F311880820A5
:104BE000FFF700FF002383F3118808BD49B1064B8E
:104BF00042681B6918605A60136043600420FFF725
:104C0000F1BE4FF0FF307047E8350020036898424E
:104C100006D01A680260506059611846FFF798BEC6
:104C20007047000038B504460D462068844200D124
:104C300038BD036823605C604561FFF789FEF4E7D7
:104C4000054B03F11402C3E905224FF0FF310022A6
:104C5000C3E90712704700BFE835002070B51C4E4D
:104C6000C0E9032305460C4601F08EFA334653F89B
:104C7000142F9A420DD13062C5E901242A600A2C12
:104C80002CBF00190A30C6E90555BDE8704001F097
:104C900069BA316A431AE31838BF1C469368A342C5
:104CA00002D9081901F06CFA73699A6894420CD819
:104CB0005A68AC602B606A6015609A685D60121B70
:104CC0009A604FF0FF33F36170BD1B68A41AECE7E4
:104CD000E835002038B51B4C636998420DD0D0E907
:104CE000003213605A6000228168C2609A680A44E8
:104CF0009A604FF0FF33E36138BD2246036842F803
:104D0000143F002193425A60C16003D1BDE838408E
:104D100001F030BA9A688168256A0A449A6001F005
:104D200033FA63699A68411B8A42E5D9AB181D1AA8
:104D3000092D206A98BF01F10A02BDE838401044ED
:104D400001F01EBAE83500202DE9F041184C00278B
:104D500004F11406656901F017FA236AAA68C11AFA
:104D60008A4215D813442362D5E9003213605A6091
:104D70006369D5F80C80EF60B34201D101F0FAF914
:104D800087F311882869C047202383F31188E1E75E
:104D90006169B14209D013441B1ABDE8F0410A2BE6
:104DA0002CBFC0180A3001F0EBB9BDE8F08100BF9C
:104DB000E83500200C2303604FF0FF3070470000FF
:104DC00000207047FEE70000704700004FF0FF3002
:104DD0007047000002290CD0032904D0012907489C
:104DE00018BF00207047032A05D8054800EBC20011
:104DF0007047044870470020704700BFF86B0008F8
:104E000040110020AC6B000870B59AB0054608460A
:104E100001A9144600F0C2F801A8FCF763FD431C89
:104E20005B00C5E900340022237003236370C6B21F
:104E300001AB02341046D1B28E4204F1020401D813
:104E40001AB070BD13F8011B04F8021C04F8010C21
:104E50000132F0E708B5202383F311880348FFF7F8
:104E60005FFA002383F3118808BD00BF603700207C
:104E700090F85C3003F01F02012A07D190F85D2002
:104E80000B2A03D10023C0E9143315E003F06003BB
:104E9000202B08D1B0F860302BB990F85D20212A82
:104EA00003D81F2A04D8FFF71DBA222AEBD0FAE74D
:104EB000034A02650722426583650120704700BFEF
:104EC0003711002007B5052917D8DFE801F01916BA
:104ED00003191920202383F31188104A019001211E
:104EE000FFF7C2FA01980E4A0221FFF7BDFA0D48FA
:104EF000FFF7E2F9002383F3118803B05DF804FBA8
:104F0000202383F311880748FFF7ACF9F2E7202349
:104F100083F311880348FFF7C3F9EBE74C6B0008F4
:104F2000706B00086037002038B50C4D0C4C0D49F3
:104F30002A4604F10800FFF767FF05F1CA0204F1F1
:104F400010000949FFF760FF05F5CA7204F1180067
:104F50000649BDE83840FFF757BF00BF283C002096
:104F6000401100202C6B0008366B0008416B0008D4
:104F700070B5044608460D46FCF7B4FCC6B22046A0
:104F8000013403780BB9184670BD32462946FCF748
:104F900095FC0028F3D10120F6E700002DE9F84F39
:104FA00005460C46FCF79EFC2B49C6B22846FFF787
:104FB000DFFF08B10436F6B228492846FFF7D8FFCC
:104FC00008B11036F6B2632E0DD8DFF88C90DFF8FA
:104FD0008CA0DFF89480DFF894B0214F2E7846B98A
:104FE0002670BDE8F88F29462046BDE8F84F01F04D
:104FF000E5BC252E2CD1072249462846FCF75EFC4D
:1050000050B93B6823607B6863603B892381BB7A2E
:10501000A37207350B34E1E7082251462846FCF716
:105020004DFCA8B90F4BA21C19780909023211F8DE
:10503000081002F8041C13F8011B01F00F015B4576
:1050400011F8081002F8031CEED118340835C5E732
:1050500004F8016B0135C1E7186C0008416B0008CA
:10506000FA6900089075FF1F206C00089C75FF1FEF
:10507000BFF34F8F024A1369DB03FCD4704700BFB4
:105080000020024008B5094B1B7873B9FFF7F0FF09
:10509000074B5A69002ABFBF064A9A6002F188325C
:1050A0009A601A6822F480621A6008BD983E002057
:1050B000002002402301674508B50B4B1B7893B9CC
:1050C000FFF7D6FF094B5A6942F000425A611A684D
:1050D00042F480521A601A6822F480521A601A68E8
:1050E00042F480621A6008BD983E00200020024011
:1050F0007F289ABF00F58030C00200207047000072
:105100004FF4006070470000802070477F2808B58A
:105110000BD8FFF7EDFF00F500630268013204D100
:1051200004308342F9D1012008BD0020FCE70000D3
:105130007F2838B5044626D8FFF7EAFCFFF798FF2A
:10514000FFF7A0FF114BF3221A6102225A615A693C
:1051500042EAC4025A615A6942F480325A610546F1
:105160002046FFF785FF4FF40061FFF7C1FF00F015
:1051700049F92846FFF7A0FFFFF7D4FC2046BDE819
:105180003840FFF7C3BF002038BD00BF00200240F9
:1051900040EA020313F007032DE9F04705460C46E9
:1051A000164606D0324B40F2FB221A600020BDE8C2
:1051B000F08781182F4A91420CD92D4A4FF4407143
:1051C0001160F3E72B1D1B686268934208D1083E0B
:1051D00008350834072E19D92A6823689A42F1D075
:1051E000FFF796FCFFF74EFFFFF742FF04F10801BF
:1051F000214C4FF001084FF00009012EA1F10807E2
:1052000008D8FFF759FFFFF78DFC01E0002EE7D12A
:105210000120CCE7C4F81480AA4651F8083C4AF8AB
:10522000043B51F8043C6B60FFF722FFC4F8149074
:105230002A6851F8083C9A420ED00D4B40F22632B3
:105240001A600E4B1D600E4B1E600E4B1F60FFF769
:1052500033FFFFF767FCA9E7DAF800A051F8043C38
:105260009A4501F10801E8D1083E0835C5E700BFBD
:10527000943E00200000040800200240883E0020E8
:10528000903E00208C3E0020084908B50B7828B1DC
:105290001BB9FFF7F7FE01230B7008BD002BFCD0F4
:1052A000BDE808400870FFF707BF00BF983E002028
:1052B0004FF4A0214FF0005000F0A6B870B582B0B6
:1052C000FFF726FC0E4E054600F05EFF3268904266
:1052D00037BF0C4A0B49516814682EBFD1E9004111
:1052E000013151600419034641F100012846019142
:1052F0003360FFF717FC0199204602B070BD00BF74
:105300009C3E0020A03E002070B582B0FFF700FC5C
:10531000104E054600F038FF3268904237BF0E4A03
:105320000D49516814682EBFD1E900410131516027
:10533000041941F100010346284601913360FFF74B
:10534000F1FB01994FF47A7200232046FAF740FFEF
:1053500002B070BD9C3E0020A03E002010B502446B
:10536000064BD2B2904200D110BD441C00B253F89B
:10537000200041F8040BE0B2F4E700BF50280040E1
:10538000114B30B5D3F89040240409D4D3F89040A1
:10539000C3F89040D3F8904044F40044C3F89040E0
:1053A0000A4C236843F4807323600244084BD2B252
:1053B000904200D130BD441C00B251F8045B43F868
:1053C0002050E0B2F4E700BF00100240007000403F
:1053D0005028004007B5012201A90020FFF7BEFFB9
:1053E000019803B05DF804FB13B50446FFF7F2FF24
:1053F000A04205D0012201A900200194FFF7C0FFBF
:1054000002B010BD704700007047000070470000F8
:10541000034B1B781BB1034B4AF6AA221A60704754
:10542000AC3E002000300040054B1A6832B902F152
:10543000804202F50432D2F894201A60704700BF0F
:10544000A83E0020024B4FF40002C3F8942070479E
:105450000010024008B5FFF7E7FF024B1868C0F3E1
:10546000407008BDA83E002070470000FEE7000025
:105470000A4B0B480B4A90420BD30B4BDA1C121A07
:10548000C11E22F003028B4238BF00220021FCF72C
:1054900031BA53F8041B40F8041BECE7146E000803
:1054A000D43F0020D43F0020D43F002070470000AC
:1054B00070B5D0E91B439E6800224FF0FF3504EB26
:1054C00042135101D3F800090028BEBFD3F80009E8
:1054D00040F08040C3F80009D3F8000B0028BEBF9D
:1054E000D3F8000B40F08040C3F8000B0132631882
:1054F0009642C3F80859C3F8085BE0D24FF0011395
:10550000C4F81C3870BD00001D4B03EB80022DE970
:10551000F043D2F80CC0DD6EDCF81420461CD2F843
:1055200000E005EB063605EB4018516871450AD3DB
:10553000D5F83438012202FA00F023EA0000C5F859
:105540003408BDE8F083BCF81040AEEB0103A34281
:1055500028BF2346D8F81849A4B2B3EB840FF0D87B
:105560009468A4F1040959F8047F3760A4EB090793
:105570001F44042FF7D81C440B4494605360D4E7B5
:10558000B03E0020890141F02001016103699B06C2
:10559000FCD41220FFF7D6BA10B5054C2046FEF712
:1055A00041FF4FF0A043E366024B236710BD00BFED
:1055B000B03E0020586C000870B50378012B0546FA
:1055C00050D12A4BC46E98421BD1294BDA6C42F45D
:1055D0008052DA64DA6E42F48052DA66DA6EDA6A9F
:1055E00042F48052DA62DA6A22F48052DA620E21E0
:1055F0004320DB6AFEF79EFB1E4BE3601E4BC4F8A4
:1056000000380023C4F8003EC0232360EE6E4FF440
:105610000413A3633369002BFCDA012333610C20EC
:10562000FFF790FA3369DB07FCD41220FFF78AFA00
:105630003369002BFCDA0026A6602846FFF738FF06
:105640006B68C4F81068DB68C4F81468C4F81C6898
:105650004BB90A4BA3614FF0FF336361A36843F07A
:105660000103A36070BD064BF4E700BFB03E00200D
:10567000001002404014004003002002003C30C0F3
:10568000083C30C0F8B5C46E054600212046FFF73F
:1056900079FF296F00234FF001128F68C4F8343866
:1056A0004FF00066C4F81C284FF0FF3004EB4312A3
:1056B00001339F42C2F80069C2F8006BC2F80809C2
:1056C000C2F8080BF2D20B68EA6E6B6763621023B4
:1056D0001361166916F01006FBD11220FFF732FA9B
:1056E000D4F8003823F4FE63C4F80038A36943F407
:1056F000402343F01003A3610923C4F81038C4F811
:1057000014380A4BEB604FF0C043C4F8103B084B11
:10571000C4F8003BC4F81069C4F800396B6F03F19A
:10572000100243F480136A67A362F8BD346C00086A
:1057300040800010C26E90F86610D2F8003823F452
:10574000FE6343EA0113C2F8003870472DE9F843BD
:1057500000EB8103C56EDA68166806F00306731E57
:10576000022B05EB41130C4680460FFA81F94FEAF4
:1057700041104FF00001C3F8101B4FF0010104F17C
:10578000100398BFB60401FA03F391698EBF334E3C
:1057900006F1805606F5004600293AD0578A04F1F2
:1057A0005801490137436F50D5F81C180B43C5F811
:1057B0001C382B180021C3F8101953690127611EEA
:1057C000A7409BB3138A928B9B08012A88BF53433F
:1057D000D8F87420981842EA034301F1400205EB1F
:1057E0008202C8F87400214653602846FFF7CAFEBB
:1057F00008EB8900C3681B8A43EA84534834640178
:105800001E432E51D5F81C381F43C5F81C78BDE83F
:10581000F88305EB4917D7F8001B21F40041C7F8BE
:10582000001BD5F81C1821EA0303C0E704F13F036D
:1058300005EB83030A4A5A6028462146FFF7A2FE79
:1058400005EB4910D0F8003923F40043C0F80039C3
:10585000D5F81C3823EA0707D7E700BF00800010FF
:1058600000040002026F12684267FFF721BE0000C9
:105870005831C36E49015B5813F4004004D013F44F
:10588000001F0CBF02200120704700004831C36E8A
:1058900049015B5813F4004004D013F4001F0CBFFF
:1058A000022001207047000000EB8101CB68196ADB
:1058B0000B6813604B6853607047000000EB810376
:1058C00030B5DD68AA691368D36019B9402B84BF6D
:1058D000402313606B8A1468C26E1C44013CB4FB05
:1058E000F3F46343033323F0030302EB411043EA71
:1058F000C44343F0C043C0F8103B2B6803F00303DC
:10590000012B09B20ED1D2F8083802EB411013F482
:10591000807FD0F8003B14BF43F0805343F0005326
:10592000C0F8003B02EB4112D2F8003B43F00443C5
:10593000C2F8003B30BD00002DE9F041244DEE6E71
:1059400006EB40130446D3F8087BC3F8087B3807FE
:105950000AD5D6F81438190706D505EB8403214675
:10596000DB6828465B689847FA071FD5D6F81438D5
:10597000DB071BD505EB8403D968CCB98B69488A52
:105980005A68B2FBF0F600FB16228AB91868DA688A
:1059900090420DD2121AC3E90024202383F3118808
:1059A0000B482146FFF78AFF84F31188BDE8F08198
:1059B000012303FA04F26B8923EA02036B81CB68AB
:1059C000002BF3D021460248BDE8F041184700BF44
:1059D000B03E002000EB810370B5DD68C36E6C69DA
:1059E0002668E6604A0156BB1A444FF40020C2F80C
:1059F00010092A6802F00302012A0AB20ED1D3F874
:105A0000080803EB421410F4807FD4F8000914BF97
:105A100040F0805040F00050C4F8000903EB4212FF
:105A2000D2F8000940F00440C2F80009D3F8340865
:105A3000012202FA01F10143C3F8341870BD19B90B
:105A4000402E84BF4020206020682E8A8419013CAB
:105A5000B4FBF6F440EAC44040F000501A44C6E7F4
:105A6000F8B504461E48C56E05EB4413D3F8086923
:105A7000C3F80869F10717D5D5F81038DA0713D538
:105A800000EB8403D9684B691F68DA68974218D223
:105A9000D21B00271A605F60202383F31188214600
:105AA000FFF798FF87F31188330617D5D5F8342808
:105AB0000123A340134211D02046BDE8F840FFF770
:105AC00023BD012303FA04F2038923EA02030381BD
:105AD0008B68002BE8D021469847E5E7F8BD00BF6A
:105AE000B03E00202DE9F74FA34CE66E7569B3690F
:105AF0001D4015F48058756107D02046FEF7FEFC66
:105B000003B0BDE8F04FFDF7DFBF002D12DAD6F885
:105B1000003E99489F071EBFD6F8003E23F00303BE
:105B2000C6F8003ED6F8043823F00103C6F804385E
:105B3000FEF70EFD280505D58F48FFF7B9FC8E4806
:105B4000FEF7F6FCA9040CD5D6F8083813F0060FBA
:105B5000F36823F470530CBF43F4105343F4A05381
:105B6000F3602A0704D56368DB680BB18248984765
:105B7000EB0200F18A80AF0227D5D4F86C90DFF8F1
:105B8000F8B100274FF0010A09EB4712D2F8003BA9
:105B900003F44023B3F5802F11D1D2F8003B002B42
:105BA0000DDA62890AFA07F322EA0303638104EB40
:105BB0008703DB68DB6813B1394658469847236F83
:105BC00001379B68FFB29F42DED9E80618D5E76E21
:105BD0003A6AC2F30A1002F00F0302F4F012B2F5AF
:105BE000802F00F09D80B2F5402F09D104EB830394
:105BF0000022DB681B6A07F58057904240F08280E4
:105C00002B03D6F818481DD5E70302D50020FFF76F
:105C100093FEA60302D50120FFF78EFE600302D596
:105C20000220FFF789FE210302D50320FFF784FE3F
:105C3000E20202D50420FFF77FFEA30202D5052071
:105C4000FFF77AFE6F037FF55BAFE60702D5002012
:105C5000FFF706FFA50702D50120FFF701FF600748
:105C600002D50220FFF7FCFE210702D50320FFF733
:105C7000F7FEE20602D50420FFF7F2FEA3067FF549
:105C80003FAF0520FFF7ECFE3AE7E36EDFF8E8B040
:105C9000019300274FF0010A236F9B685FFA87F991
:105CA00099453FF668AF019B03EB4913D3F80029F0
:105CB00002F44022B2F5802F22D1D3F80029002A25
:105CC0001EDAD3F8002942F09042C3F80029D3F835
:105CD0000029002AFBDBE06E4946FFF753FC2289CE
:105CE0000AFA09F322EA0303238104EB8903DB6840
:105CF0009B6813B14946584698474846FFF704FC4D
:105D00000137C9E7910708BFD7F80080072A98BF75
:105D100003F8018B02F1010298BF4FEA18286CE7E3
:105D2000023304EB830207F580575268D2F818C09B
:105D3000DCF80820DCE9001CA1EB0C0C00218842F7
:105D40000AD104EB830463689B699A6802449A60F1
:105D50005A6802445A6053E711F0030F08BFD7F89E
:105D600000808C4588BF02F8018B01F1010188BFDA
:105D70004FEA1828E3E700BFB03E0020C36E03EBF4
:105D80004111D1F8003B43F40013C1F8003B7047C8
:105D9000C36E03EB4111D1F8003943F40013C1F88D
:105DA00000397047C36E03EB4111D1F8003B23F477
:105DB0000013C1F8003B7047C36E03EB4111D1F8EB
:105DC000003923F40013C1F80039704730B5039C43
:105DD0000172043304FB0325C0E90653049B0363EB
:105DE0000021059BC160C0E90000C0E90422C0E9B0
:105DF0000842C0E90A11436330BD0000416A002235
:105E0000C0E90411C0E90A22C2606FF00101FEF787
:105E100009BF0000D0E90432934201D1C2680AB937
:105E2000181D70470020704703691960C26801326D
:105E3000C260C269134482690361934224BF436A0A
:105E400003610021FEF7E2BE38B504460D46E36863
:105E50003BB16269131D1268A3621344E362002020
:105E600007E0237A33B929462046FEF7BFFE002813
:105E7000EDDA38BD6FF00100FBE70000C368C269CE
:105E8000013BC3604369134482694361934224BF69
:105E9000436A436100238362036B03B11847704771
:105EA00070B52023044683F31188866A3EB9FFF754
:105EB000CBFF054618B186F31188284670BDA36A4A
:105EC000E26A13F8015BA362934202D32046FFF714
:105ED000D5FF002383F31188EFE700002DE9F84F89
:105EE00004460E46174698464FF0200989F311885C
:105EF0000025AA46D4F828B0BBF1000F09D14146CD
:105F00002046FFF7A1FF20B18BF311882846BDE89A
:105F1000F88FD4E90A12A7EB050B521A934528BF54
:105F20009346BBF1400F1BD9334601F1400251F8B3
:105F3000040B43F8040B9142F9D1A36A4033403675
:105F4000A3624035D4E90A239A4202D32046FFF7E0
:105F500095FF8AF31188BD42D8D289F31188C9E729
:105F600030465A46FBF7A0FCA36A5B445E44A3623A
:105F70005D44E7E710B5029C0172043304FB032182
:105F8000C0E906130023C0E90A33039B0363049BA3
:105F9000C460C0E90000C0E90422C0E908424363CC
:105FA00010BD0000026AC260426AC0E904220022F9
:105FB000C0E90A226FF00101FEF734BED0E90423E4
:105FC0009A4201D1C26822B9184650F8043B0B60CE
:105FD0007047002070470000C368C2690133C36086
:105FE0004369134482694361934224BF436A436116
:105FF0000021FEF70BBE000038B504460D46E368ED
:106000003BB123691A1DA262E2691344E3620020D6
:1060100007E0237A33B929462046FEF7E7FD00283A
:10602000EDDA38BD6FF00100FBE70000036919608D
:10603000C268013AC260C269134482690361934233
:1060400024BF436A036100238362036B03B11847D3
:106050007047000070B520230D460446114683F3B7
:106060001188866A2EB9FFF7C7FF10B186F3118831
:1060700070BDA36A1D70A36AE26A01339342A362F2
:1060800004D3E16920460439FFF7D0FF002080F3F4
:106090001188EDE72DE9F84F04460D4690469946E4
:1060A0004FF0200A8AF311880026B346A76A4FB939
:1060B00049462046FFF7A0FF20B187F311883046FC
:1060C000BDE8F88FD4E90A073A1AA8EB0607974209
:1060D00028BF1746402F1BD905F1400355F8042B64
:1060E00040F8042B9D42F9D1A36A4033A3624036A5
:1060F000D4E90A239A4204D3E16920460439FFF720
:1061000095FF8BF311884645D9D28AF31188CDE7E4
:1061100029463A46FBF7C8FBA36A3B443D44A362C9
:106120003E44E5E7D0E904239A4217D1C3689BB106
:10613000836A8BB1043B9B1A0ED01360C368013B8A
:10614000C360C3691A44836902619A4224BF436AE7
:106150000361002383620123184670470023FBE795
:1061600000F080B84FF08043002258631A61022289
:10617000DA6070474FF080430022DA607047000019
:106180004FF08043586370474FF08043586A704720
:106190004B6843608B688360CB68C3600B69436165
:1061A0004B6903628B6943620B68036070470000B0
:1061B00008B5234BDA6A42F0FF02DA62DA6A22F0AB
:1061C000FF02DA62DA6ADA6C42F0FF02DA64DA6E4F
:1061D00042F0FF02DA661B4ADB6E11464FF0904038
:1061E000FFF7D6FF02F11C0100F58060FFF7D0FF3A
:1061F00002F1380100F58060FFF7CAFF02F1540197
:1062000000F58060FFF7C4FF02F1700100F58060C7
:10621000FFF7BEFF02F18C0100F58060FFF7B8FFC9
:1062200002F1A80100F58060FFF7B2FF02F1C4019E
:1062300000F58060FFF7ACFFBDE8084000F09EB8B5
:1062400000100240646C000808B500F023FAFEF765
:1062500031FCFFF7E9F8BDE80840FEF765BE000035
:10626000704700000F4B9A6D42F001029A659A6FD9
:1062700042F001029A670C4A9B6F936843F0010356
:1062800093604FF080434F229A624FF0FF32DA6200
:1062900000229A615A63DA605A6001225A611A60D8
:1062A000704700BF00100240002004E04FF0804221
:1062B00008B51169D3680B40D9B2C9439B07116176
:1062C00007D5202383F31188FEF720FC002383F3F6
:1062D000118808BD08B5274B4FF0FF319A6A9962C3
:1062E0009A6A00229A62986AD86A60F0FF00D862BF
:1062F000D86AC0B2D862D86A186B1963186B1A636F
:10630000186B986B60F080509863986B00F0805029
:106310009863986BD86BD963D86BDA63D86B186CB9
:106320001964196C1A64196C996D41F08051996562
:10633000996F41F080519967996FD3F8901011F4DB
:10634000407F1EBF4FF48031C3F89010C3F89020F7
:10635000D3F89020C3F8902000F074F9064B002287
:106360005A605A6842F480625A605A6842F4007275
:106370005A6008BD00100240007000403A4B3B4A92
:106380009A6501221A601A689007FCD500229A606B
:106390009A6812F00C0FFBD1354A4FF4007111606E
:1063A00051694905FCD41A6842F480721A601A686F
:1063B0005205FCD52E490A6842F480720A602D4AC3
:1063C0004FF4E06111601A6842F060021A601A68C6
:1063D00042F008021A601A689007FCD59A6812F019
:1063E0000C0FFBD1D3F8942042F4C062C3F8942080
:1063F000214ADA601A6842F080721A601A689101C4
:10640000FCD51E4A1A611A6842F080621A601A6846
:106410001201FCD500229A60194AC3F88820154958
:106420000122C3F89C200A6822F0070242F004020D
:106430000A600A6802F00702042AFAD19A6842F058
:1064400003029A609A6802F00C020C2AFAD11A6EC2
:1064500042F001021A66D3F8802042F00102C3F82C
:106460008020D3F8803070470010024000040010F4
:10647000007000400020024012140001000C1000C7
:1064800055550134074A08B5536903F001035361B8
:1064900023B1054A13680BB150689847BDE808401E
:1064A000FDF712BB00040140403F0020074A08B539
:1064B000536903F00203536123B1054A93680BB19A
:1064C000D0689847BDE80840FDF7FEBA00040140D7
:1064D000403F0020074A08B5536903F004035361A5
:1064E00023B1054A13690BB150699847BDE80840CC
:1064F000FDF7EABA00040140403F0020074A08B512
:10650000536903F00803536123B1054A93690BB142
:10651000D0699847BDE80840FDF7D6BA00040140AD
:10652000403F0020074A08B5536903F01003536148
:1065300023B1054A136A0BB1506A9847BDE8084079
:10654000FDF7C2BA00040140403F0020164B10B5D1
:106550005C6904F478725A61A30604D5134A936AFD
:106560000BB1D06A9847600604D5104A136B0BB183
:10657000506B9847210604D50C4A936B0BB1D06B36
:106580009847E20504D5094A136C0BB1506C984743
:10659000A30504D5054A936C0BB1D06C9847BDE8B0
:1065A0001040FDF791BA00BF00040140403F0020B9
:1065B000194B10B55C6904F47C425A61620504D53C
:1065C000164A136D0BB1506D9847230504D5134A35
:1065D000936D0BB1D06D9847E00404D50F4A136E4C
:1065E0000BB1506E9847A10404D50C4A936E0BB1C1
:1065F000D06E9847620404D5084A136F0BB1506FF0
:106600009847230404D5054A936F0BB1D06F984780
:10661000BDE81040FDF758BA00040140403F00209B
:1066200008B50348FDF702FBBDE80840FDF74CBA8A
:106630003C35002008B5FFF739FEBDE80840FDF7FE
:1066400043BA0000062108B50846FDF773FB062192
:106650000720FDF76FFB06210820FDF76BFB0621E5
:106660000920FDF767FB06210A20FDF763FB0621E1
:106670001720FDF75FFB06212820FDF75BFB0721B4
:106680001C20FDF757FBBDE808400C212520FDF735
:1066900051BB000008B5FFF71DFE00F00DF8FDF737
:1066A000EDFCFDF7BDFEFDF795FDFFF7D9FDBDE85B
:1066B0000840FFF755BD00000023054A1946013385
:1066C000102BC2E9001102F10802F8D1704700BF97
:1066D000403F00200B460146184600F025B8000058
:1066E00000F038B8012838BF012010B50446204614
:1066F00000F028F830B900F007F808B900F00CF8FD
:106700008047F4E710BD0000024B1868BFF35B8FB1
:10671000704700BFC03F002008B5062000F032F9E6
:106720000120FEF74FFB000010B5054C13462CB1BD
:106730000A4601460220AFF3008010BD2046FCE768
:1067400000000000024B0146186800F089B800BF45
:1067500060110020024B0146186800F035B800BFF8
:106760006011002010B501390244904201D100208F
:1067700005E0037811F8014FA34201D0181B10BDAA
:106780000130F2E72DE9F041A3B1C91A17780144AD
:10679000044603F1FF3C8C42204601D9002009E069
:1067A0000578BD4204F10104F5D10CEB0405D618BF
:1067B000A54201D1BDE8F08115F8018D16F801ED73
:1067C000F045F5D0E7E7000037B5002944D051F88F
:1067D000043C0190002BA1F10404B8BFE41800F0C0
:1067E000F5F81E4A0198136833B96360146003B06A
:1067F000BDE8304000F0F0B8A34208D9256861191F
:106800008B4201BF19685B6849192160EDE71A46A0
:106810005B680BB1A342FAD911685518A5420BD198
:10682000246821445418A3421160E0D11C685B68BD
:10683000536021441160DAE702D90C230360D6E7E4
:10684000256861198B4204BF19685B68636004BFE7
:10685000491921605460CAE703B030BDC43F00202D
:10686000F8B5CD1C25F0030508350C2D38BF0C25D7
:10687000002D064601DBA94203D90C23336000201A
:10688000F8BD00F0A3F821490A6814469CB9204FCE
:106890003B6823B92146304600F03CF83860294671
:1068A000304600F037F8431C23D10C2333603046C8
:1068B00000F092F8E3E723685B1B17D40B2B03D996
:1068C00023601C44256004E06368A2420CBF0B6097
:1068D0005360304600F080F804F10B00231D20F0D7
:1068E0000700C21ACCD01B1AA350C9E7224664681D
:1068F000CCE7C41C24F00304A042E3D0211A3046A4
:1069000000F008F80130DDD1CFE700BFC43F002020
:10691000C83F002038B5064D0023044608462B60CA
:10692000FEF748FA431C02D12B6803B1236038BD3F
:10693000CC3F00201F2938B504460D4604D9162344
:1069400003604FF0FF3038BD426C12B152F8213075
:106950004BB9204600F030F82A4601462046BDE8F3
:10696000384000F017B8012B0AD0591C03D1162368
:1069700003600120E7E7002442F8254028469847B5
:106980000020E0E7024B01461868FFF7D3BF00BFC5
:106990006011002038B5074D002304460846114613
:1069A0002B60FEF713FA431C02D12B6803B123605E
:1069B00038BD00BFCC3F0020FEF702BA034611F8F5
:1069C000012B03F8012B002AF9D17047014800F090
:1069D00009B800BFD03F0020014800F005B800BF53
:1069E000D03F002070470000704700006F72672E94
:1069F0006172647570696C6F742E4E75636C656F2F
:106A00002D4C34393600000053544D33324C343F52
:106A10003F0000004261642043414E496661636566
:106A200020696E6465782E00800000000080000000
:106A30000000800000000000000000007D1A000837
:106A400065220008C52100088D1A0008C11A000837
:106A5000BD1C0008911A0008A11A0008951A000828
:106A60009D1A0008991A0008E51B0008A51A0008DD
:106A7000D1240008B51A0008B91B000840A2E4F1AF
:106A8000646891060041A3E5F26569920700000081
:106A90000096000000000000000000000000000060
:106AA0000000000000000000000000004540000859
:106AB000314000086D40000859400008654000085A
:106AC000514000083D400008294000087940000876
:106AD00000000000514100083D41000879410008D4
:106AE00065410008714100085D4100084941000806
:106AF0003541000885410008000000000100000049
:106B0000000000006D61696E0000000069646C6542
:106B1000000000000C6B00082836002060370020C1
:106B200001000000B14A00080000000041726475D5
:106B300050696C6F740025424F415244252D424CE0
:106B4000002553455249414C250000000200000039
:106B5000000000006D430008D943000840004000D9
:106B6000F83B0020083C002002000000000000006C
:106B700003000000000000001D44000800000000A9
:106B800010000000183C0020000000000100000080
:106B900000000000B03E002001010200C54E0008C8
:106BA000D54D0008714E0008554E00084300000006
:106BB000B46B000809024300020100C0320904005E
:106BC000000102020100052400100105240100015A
:106BD000042402020524060001070582030800FFC1
:106BE00009040100020A000000070501024000003C
:106BF000070581024000000012000000006C000840
:106C00001201100102000040091241570002010266
:106C1000030100000403090425424F4152442500AA
:106C200030313233343536373839414243444546C2
:106C30000000000000000000654500081D48000835
:106C4000C948000840004000283F0020283F00209D
:106C500001000000383F00208000000040010000DB
:106C6000050000000000A82A00000000AAAABEAA91
:106C700000001424FFFF00000000000070A70A00BD
:106C80000040001000000000AAAAAAAA000000000C
:106C90007FBF0000000000000000000000000000B6
:106CA00000000000AAAAAAAA00000000FFFF00003E
:106CB00000000000000000000A00000000000000CA
:106CC000AAAAAAAA00000000FFFF00009900000085
:106CD000000000000000000000000000AAAAAAAA0C
:106CE00000000000FFFF00000000000000000000A6
:106CF0000000000000000000AAAAAAAA00000000EC
:106D0000FFFF000000000000000000000000000085
:106D100000000000AAAAAAAA00000000FFFF0000CD
:106D20000000000000000000000000000000000063
:106D3000AAAAAAAA00000000FFFF000000000000AD
:106D400000000000BC94FF7F010000000000000074
:106D500017040000000000000060030000000000B5
:106D6000FE2A0100D2040000FF000000603700206E
:106D70003C35002000000000086A00083F000000C9
:106D800000960000000008009600000000080000C7
:106D900004000000146C0008000000000000000067
:106DA00000000000000000000000000000000000E3
:106DB000641100200000000000000000000000003E
:106DC00000000000000000000000000000000000C3
:106DD00000000000000000000000000000000000B3
:106DE00000000000000000000000000000000000A3
:106DF0000000000000000000000000000000000093
:106E00000000000000000000000000000000000082
:046E1000000000007E
:00000001FF
